:020000040000FA
:0408000098EF0BF072
:1008100003B275EF05F0F2B493EF05F09EB09BEFD5
:1008200005F09EB2A3EF05F0F2A81AEF04F0F2B2C1
:1008300023EF04F0F2B01FEF04F047EF0BF0F29655
:10084000F29047EF0BF0CD90F2929EA02DEF04F0C6
:100850000101533F2DEF04F0542BB2C1B6F1B3C1E7
:10086000B7F1B4C1B8F1B5C1B9F1AEC1B2F1AFC120
:10087000B3F1B0C1B4F1B1C1B5F1AAC1AEF1ABC130
:10088000AFF1ACC1B0F1ADC1B1F1A6C1AAF1A7C140
:10089000ABF1A8C1ACF1A9C1ADF1A2C1A6F1A3C150
:1008A000A7F1A4C1A8F1A5C1A9F19EC1A2F19FC160
:1008B000A3F1A0C1A4F1A1C1A5F19AC19EF19BC170
:1008C0009FF19CC1A0F19DC1A1F1CECF9AF1CFCFF4
:1008D0009BF153C19CF154C19DF1CF6ACE6A0101D5
:1008E000536B546B9E90CD800FBC0F8E0FBA7CEF74
:1008F00004F00F8A47EF0BF013880F8C0FBEB9EF8F
:1009000004F09AC19EF19BC19FF19CC1A0F19DC1D1
:10091000A1F19EC1A2F19FC1A3F1A0C1A4F1A1C107
:10092000A5F1A2C1A6F1A3C1A7F1A4C1A8F1A5C1D7
:10093000A9F1A6C1AAF1A7C1ABF1A8C1ACF1A9C1A7
:10094000ADF1AAC1AEF1ABC1AFF1ACC1B0F1ADC177
:10095000B1F1AEC1B2F1AFC1B3F1B0C1B4F1B1C147
:10096000B5F1B2C1B6F1B3C1B7F1B4C1B8F1B5C117
:10097000B9F101015E6B5F6B606B616B9A515E2731
:100980009B515F239C5160239D5161239E515E27A3
:100990009F515F23A0516023A1516123A2515E2783
:1009A000A3515F23A4516023A5516123A6515E2763
:1009B000A7515F23A8516023A9516123AA515E2743
:1009C000AB515F23AC516023AD516123AE515E2723
:1009D000AF515F23B0516023B1516123B2515E2703
:1009E000B3515F23B4516023B5516123B6515E27E3
:1009F000B7515F23B8516023B9516123D8900101E9
:100A0000613360335F335E33D8900101613360330B
:100A10005F335E33D8900101613360335F335E33FF
:100A200000C10CF101C10DF102C10EF103C10FF1C2
:100A300004C110F105C111F106C112F107C113F192
:100A400008C114F109C115F10AC116F10BC117F162
:100A500034C135F111B838EF05F00101620E046FB1
:100A6000010E056F000E066F000E076F41EF05F0D7
:100A70000101A70E046F020E056F000E066F000E37
:100A8000076F5EC100F15FC101F160C102F161C198
:100A900003F1FDEC30F003BF04D01CBE02D01CA05B
:100AA000108C11A059EF05F010BA59EF05F00F8026
:100AB000108A0CC100F10DC101F10EC102F10FC18C
:100AC00003F110C104F111C105F112C106F113C106
:100AD00007F114C108F115C109F116C10AF117C1D6
:100AE0000BF135C134F147EF0BF00392ABB2AB9889
:100AF000AB88030103EE00F080517F0BE92604C0B0
:100B0000EFFF802B8151805D700BD8A48B82000099
:100B10008051815D700BD8A48B9281518019D8B41B
:100B2000079047EF0BF0F2940101453F47EF0BF0C0
:100B3000462B47EF0BF09E900101533F47EF0BF020
:100B4000542B47EF0BF09E9211B843EF08F00400CE
:100B500066A1ABEF05F08BB4B5EF05F010ACB5EFC7
:100B600005F08B84109CB6EF05F08B94077C07ACE6
:100B7000D1EF05F0C274C2B4CBEF05F0C3CFB7F527
:100B8000C4CFB8F50501D890B833B733D890B8338F
:100B9000B733D2EF05F0C3CF55F1C4CF56F1D2EF42
:100BA00005F0C28207B444EF06F047C14BF148C1DB
:100BB0004CF149C14DF14AC14EF15EC162F15FC1D4
:100BC00063F160C164F161C165F113A8EAEF05F05A
:100BD000138C13989AC1BAF19BC1BBF19CC1BCF1B3
:100BE0009DC1BDF19EC1BEF19FC1BFF1A0C1C0F1C9
:100BF000A1C1C1F1A2C1C2F1A3C1C3F1A4C1C4F199
:100C0000A5C1C5F1A6C1C6F1A7C1C7F1A8C1C8F168
:100C1000A9C1C9F1AAC1CAF1ABC1CBF1ACC1CCF138
:100C2000ADC1CDF1AEC1CEF1AFC1CFF1B0C1D0F108
:100C3000B1C1D1F1B2C1D2F1B3C1D3F1B4C1D4F1D8
:100C4000B5C1D5F1B6C1D6F1B7C1D7F1B8C1D8F1A8
:100C5000B9C1D9F1B7C5B9F5B8C5BAF5B9C5BBF5CC
:100C6000BAC5BCF5010155515B2756515C23E86AB2
:100C70005D230E2E44EF06F05CC157F15DC158F1C3
:100C80005B6B5C6B5D6B078E0201002F47EF0BF017
:100C90003C0E006F1D50E00BE00AE86612881BBE98
:100CA00002D01BB4108E00C10CF101C10DF102C1C4
:100CB0000EF103C10FF104C110F105C111F106C11C
:100CC00012F107C113F108C114F109C115F10AC1EC
:100CD00016F10BC117F134C135F181AAACEF06F062
:100CE00015A4F7EF06F005012F51000AD8B43AEF2A
:100CF00007F005012F51010AD8B4B6EF06F005013F
:100D00002F51020AD8B4F7EF06F005012F51030A5C
:100D1000D8B4F7EF06F005012F51040AD8B4F7EF65
:100D200006F005012F51050AD8B4F7EF06F00501CA
:100D30002F51060AD8B4F7EF06F005012F51070A24
:100D4000D8B4F7EF06F005012F51320AD8B4B4EF4A
:100D500006F02F6B3AEF07F000011650030AD8B4E3
:100D6000F7EF06F03AEF07F03AEF07F005015767A3
:100D7000C1EF06F05867C1EF06F05967C1EF06F002
:100D80005A67C5EF06F03AEF07F05BC500F15CC5A6
:100D900001F15DC502F15EC503F10101010E046FB1
:100DA000000E056F000E066F000E076FFDEC30F0B1
:100DB00000C15BF501C15CF502C15DF503C15EF5E3
:100DC00001010067EBEF06F00167EBEF06F0026749
:100DD000EBEF06F003673AEF07F057C55BF558C530
:100DE0005CF559C55DF55AC55EF524EF07F00FBEF9
:100DF0000CEF07F010A011EF07F00101476708EFB3
:100E000007F0486708EF07F0496708EF07F04A67FF
:100E10000CEF07F011EF07F007AE11EF07F024EF2A
:100E200007F00501312F3AEF07F03C0E316F302FFC
:100E30003AEF07F00101000E626FE00E636FA50E3E
:100E4000646F010E656F138800011650000AD8B454
:100E500032EF07F000011650030AD8B437EF07F05D
:100E60003AEF07F00001010E166E3AEF07F00001AD
:100E7000040E166E0501666B37B740EF07F066810A
:100E80000CC100F10DC101F10EC102F10FC103F15E
:100E900010C104F111C105F112C106F113C107F12E
:100EA00014C108F115C109F116C10AF117C10BF1FE
:100EB00035C134F100C10CF101C10DF102C10EF1D7
:100EC00003C10FF104C110F105C111F106C112F106
:100ED00007C113F108C114F109C115F10AC116F1D6
:100EE0000BC117F134C135F101018E677FEF07F0B7
:100EF0008F677FEF07F090677FEF07F0916783EFD1
:100F000007F0B4EF07F092C100F193C101F194C171
:100F100002F195C103F10101010E046F000E056F8E
:100F2000000E066F000E076FFDEC30F000C192F16D
:100F300001C193F102C194F103C195F10101006770
:100F4000A9EF07F00167A9EF07F00267A9EF07F023
:100F50000367B4EF07F08EC192F18FC193F190C196
:100F600094F191C195F10F80D57ED5BE6ED0D6CFCC
:100F700047F1D7CF48F145C149F1E86AE8CF4AF1D6
:100F8000138A1CBE02D01CA0108C109047C100F127
:100F900048C101F149C102F14AC103F101010A0E40
:100FA000046F000E056F000E066F000E076FFDEC5C
:100FB00030F003AF1080010154A7EBEF07F00F9A58
:100FC0000F9C0F9E0101000E5E6F600E5F6F3D0E65
:100FD000606F080E616F010147BFFBEF07F04867C4
:100FE000FBEF07F04967FBEF07F04A67FBEF07F0FD
:100FF000F28820EF08F0F2985E6B5F6B606B616BBC
:101000009A6B9B6B9C6B9D6B9E6B9F6BA06BA16B9C
:10101000A26BA36BA46BA56BA66BA76BA86BA96B4C
:10102000AA6BAB6BAC6BAD6BAE6BAF6BB06BB16BFC
:10103000B26BB36BB46BB56BB66BB76BB86BB96BAC
:10104000D76AD66A0101456B466B0CC100F10DC130
:1010500001F10EC102F10FC103F110C104F111C180
:1010600005F112C106F113C107F114C108F115C150
:1010700009F116C10AF117C10BF135C134F147EF7F
:101080000BF047EF0BF00201002FABEF0AF0D59EFB
:10109000D6CF47F1D7CF48F145C149F1E86AE8CF4B
:1010A0004AF1138AD76AD66A0101456B466BD58E21
:1010B0001D50E00BE00AE86612881BBE02D01BB48C
:1010C000108E1AAE1F8C00C10CF101C10DF102C1CE
:1010D0000EF103C10FF104C110F105C111F106C1F8
:1010E00012F107C113F108C114F109C115F10AC1C8
:1010F00016F10BC117F134C135F10FA0109A11B8D8
:101100008DEF08F00101620E046F010E056F000EF5
:10111000066F000E076F96EF08F00101A70E046F2F
:10112000020E056F000E066F000E076F47C100F13B
:1011300048C101F149C102F14AC103F1FDEC30F0AF
:1011400003BFA9EF08F01CBE02D01CA0108C11B088
:101150000F800CC100F10DC101F10EC102F10FC1F0
:1011600003F110C104F111C105F112C106F113C15F
:1011700007F114C108F115C109F116C10AF117C12F
:101180000BF135C134F102013C0E006F00C10CF1CE
:1011900001C10DF102C10EF103C10FF104C110F143
:1011A00005C111F106C112F107C113F108C114F113
:1011B00009C115F10AC116F10BC117F134C135F19E
:1011C00081BAE6EF08F015B225EF09F015A025EF7A
:1011D00009F015A470EF09F005012F51000AD8B4E9
:1011E000B3EF09F005012F51010AD8B42FEF09F030
:1011F00005012F51020AD8B470EF09F005012F51F3
:10120000030AD8B470EF09F005012F51040AD8B4CD
:1012100070EF09F005012F51050AD8B470EF09F0FD
:1012200005012F51060AD8B470EF09F005012F51BE
:10123000070AD8B470EF09F005012F51320AD8B46B
:101240002DEF09F02F6BB3EF09F000011650030AE0
:10125000D8B470EF09F0B3EF09F0B3EF09F005016E
:1012600057673AEF09F058673AEF09F059673AEFD4
:1012700009F05A673EEF09F0B3EF09F05BC500F1E2
:101280005CC501F15DC502F15EC503F10101010E0E
:10129000046F000E056F000E066F000E076FFDEC69
:1012A00030F000C15BF501C15CF502C15DF503C121
:1012B0005EF50101006764EF09F0016764EF09F072
:1012C000026764EF09F00367B3EF09F057C55BF5F8
:1012D00058C55CF559C55DF55AC55EF59DEF09F039
:1012E0000FBE85EF09F010A08AEF09F001014767F2
:1012F00081EF09F0486781EF09F0496781EF09F054
:101300004A6785EF09F08AEF09F007AE8AEF09F026
:101310009DEF09F00501312FB3EF09F03C0E316F5D
:10132000302FB3EF09F00101000E626FE00E636F22
:10133000A50E646F010E656F138800011650000A38
:10134000D8B4ABEF09F000011650030AD8B4B0EFDF
:1013500009F0B3EF09F00001010E166EB3EF09F0CA
:101360000001040E166E0501666B37B7B9EF09F080
:1013700066810CC100F10DC101F10EC102F10FC176
:1013800003F110C104F111C105F112C106F113C13D
:1013900007F114C108F115C109F116C10AF117C10D
:1013A0000BF135C134F100C10CF101C10DF102C1E5
:1013B0000EF103C10FF104C110F105C111F106C115
:1013C00012F107C113F108C114F109C115F10AC1E5
:1013D00016F10BC117F134C135F101018E67F8EF39
:1013E00009F08F67F8EF09F09067F8EF09F091675F
:1013F000FCEF09F02DEF0AF092C100F193C101F169
:1014000094C102F195C103F10101010E046F000EB8
:10141000056F000E066F000E076FFDEC30F000C187
:1014200092F101C193F102C194F103C195F101015F
:10143000006722EF0AF0016722EF0AF0026722EF4D
:101440000AF003672DEF0AF08EC192F18FC193F17C
:1014500090C194F191C195F10F80109047C100F1B6
:1014600048C101F149C102F14AC103F101010A0E6B
:10147000046F000E056F000E066F000E076FFDEC87
:1014800030F003AF1080010154A753EF0AF00F9A18
:101490000F9C0F9E0101000E5E6F600E5F6F3D0E90
:1014A000606F080E616F47C100F148C101F149C189
:1014B00002F14AC103F10101140E046F050E056F1C
:1014C000000E066F000E076FFDEC30F003AF6CEFFF
:1014D0000AF0F28891EF0AF0F2985E6B5F6B606B36
:1014E000616B9A6B9B6B9C6B9D6B9E6B9F6BA06BF8
:1014F000A16BA26BA36BA46BA56BA66BA76BA86B70
:10150000A96BAA6BAB6BAC6BAD6BAE6BAF6BB06B1F
:10151000B16BB26BB36BB46BB56BB66BB76BB86BCF
:10152000B96B0CC100F10DC101F10EC102F10FC187
:1015300003F110C104F111C105F112C106F113C18B
:1015400007F114C108F115C109F116C10AF117C15B
:101550000BF135C134F104008BB4B6EF0AF010ACD6
:10156000B6EF0AF08B84109CB7EF0AF08B94077CDF
:1015700007ACD2EF0AF0C274C2B4CCEF0AF0C3CF0A
:10158000B7F5C4CFB8F50501D890B833B733D890C4
:10159000B833B733D3EF0AF0C3CF55F1C4CF56F108
:1015A000D3EF0AF0C28207B445EF0BF047C14BF10D
:1015B00048C14CF149C14DF14AC14EF15EC162F1E1
:1015C0005FC163F160C164F161C165F113A8EBEF24
:1015D0000AF0138C13989AC1BAF19BC1BBF19CC15C
:1015E000BCF19DC1BDF19EC1BEF19FC1BFF1A0C1C3
:1015F000C0F1A1C1C1F1A2C1C2F1A3C1C3F1A4C193
:10160000C4F1A5C1C5F1A6C1C6F1A7C1C7F1A8C162
:10161000C8F1A9C1C9F1AAC1CAF1ABC1CBF1ACC132
:10162000CCF1ADC1CDF1AEC1CEF1AFC1CFF1B0C102
:10163000D0F1B1C1D1F1B2C1D2F1B3C1D3F1B4C1D2
:10164000D4F1B5C1D5F1B6C1D6F1B7C1D7F1B8C1A2
:10165000D8F1B9C1D9F1B7C5B9F5B8C5BAF5B9C5A9
:10166000BBF5BAC5BCF5010155515B2756515C234A
:10167000E86A5D230E2E45EF0BF05CC157F15DC1AA
:1016800058F15B6B5C6B5D6B078E47EF0BF002C034
:10169000E0FF005001C0D8FF1000A6B24DEF0BF0E4
:1016A0000CC0A9FF0BC0A8FFA69EA69CA684F29E14
:1016B000550EA76EAA0EA76EA682F28EA694A6B2AB
:1016C0005FEF0BF00C2A1200A96EA69EA69CA680C6
:1016D000A8500C2A120004012C0E826F96EC0EF01A
:1016E00012EC32F00C5064EC0BF0E8CF00F10C502F
:1016F00064EC0BF0E8CF01F101AF84EF0BF00101D6
:10170000FF0E026FFF0E036F9BEC31F0296790EF25
:101710000BF00401200E826F96EC0EF095EF0BF0AB
:1017200004012D0E826F96EC0EF0A5EC2FF0120046
:1017300015941596076A0F6A106A116A126A136A7D
:10174000166A0F010D0EC16E860EC06E030EC26EBC
:101750000F01680E896E130E926E080E8A6EF30EDC
:10176000936E8B6A900E946EC80E64EC0BF0E8CF0B
:10177000E8FF1098E8A0108810A805D00E0E256E7E
:101780008E0E266E04D00F0E256E8F0E266EAAECDE
:1017900032F0F5EC33F0F18EF19EFC0E64EC0BF0C0
:1017A000E8CF0BF00BA011800BA211820BA41184C7
:1017B0000BA81188C90E64EC0BF0E8CF1AF0CA0E22
:1017C00064EC0BF0E8CF1BF0CB0E64EC0BF0E8CF31
:1017D0001CF0CC0E64EC0BF0E8CF1DF0FB0E64ECBB
:1017E0000BF0E8CF37F0CE0E64EC0BF0E8CF14F03E
:1017F000CD0E64EC0BF0E8CF36F01F6A206A0E6A5B
:1018000001015B6B5C6B5D6B576B586BF29A01016E
:10181000476B486B496B4A6B4B6B4C6B4D6B4E6B1C
:101820004F6B506B516B526B456B466BD76AD66AE8
:101830000F01280ED56EF28A9D90B00ECD6E01017B
:101840005E6B5F6B606B616B626B636B646B656B34
:10185000666B676B686B696B536B546BCF6ACE6A50
:101860000F9A0F9C0F9E9D80760ECA6E9D8202017C
:101870003C0E006FCC6A160E64EC0BF0E8CF00F162
:10188000170E64EC0BF0E8CF01F1180E64EC0BF0CE
:10189000E8CF02F1190E64EC0BF0E8CF03F101017F
:1018A00003AF6DEF0CF012EC32F0160E0C6E00C1AF
:1018B0000BF04DEC0BF0170E0C6E01C10BF04DEC64
:1018C0000BF0180E0C6E02C10BF04DEC0BF0190E64
:1018D0000C6E03C10BF04DEC0BF000C18EF101C199
:1018E0008FF102C190F103C191F100C192F101C1E8
:1018F00093F102C194F103C195F11A0E64EC0BF05F
:10190000E8CF00F11B0E64EC0BF0E8CF01F11C0EE8
:1019100064EC0BF0E8CF02F11D0E64EC0BF0E8CFA5
:1019200003F1010103AFC3EF0CF012EC32F01A0E19
:101930000C6E00C10BF04DEC0BF01B0E0C6E01C1D8
:101940000BF04DEC0BF01C0E0C6E02C10BF04DECCD
:101950000BF01D0E0C6E03C10BF04DEC0BF01A0ECC
:1019600064EC0BF0E8CF00F11B0E64EC0BF0E8CF59
:1019700001F11C0E64EC0BF0E8CF02F11D0E64ECDB
:101980000BF0E8CF03F100C196F101C197F102C15C
:1019900098F103C199F1240EAC6E900EAB6E240E3B
:1019A000AC6E080EB86E000EB06E1F0EAF6E040166
:1019B000806B816B0F01900EAB6E0F019D8A03014E
:1019C000806B816BC26B8B924FEC37F04FEC37F032
:1019D00031EC39F02DEC35F0200E64EC0BF0E8CF53
:1019E0002FF505012F51FF0AD8A4FEEF0CF02F6B45
:1019F000200E0C6E2FC50BF04DEC0BF00501010E07
:101A0000306F3C0E316F250E64EC0BF0E8CF00F127
:101A1000260E64EC0BF0E8CF01F1270E64EC0BF01E
:101A2000E8CF02F1280E64EC0BF0E8CF03F10101DE
:101A300003AF35EF0DF012EC32F0250E0C6E00C145
:101A40000BF04DEC0BF0260E0C6E01C10BF04DECC3
:101A50000BF0270E0C6E02C10BF04DEC0BF0280EB4
:101A60000C6E03C10BF04DEC0BF000C157F501C13A
:101A700058F502C159F503C15AF500C15BF501C122
:101A80005CF502C15DF503C15EF5290E64EC0BF057
:101A9000E8CF5FF5050160515F5DD8A05FC560F5D7
:101AA000210E64EC0BF0E8CF00F1220E64EC0BF099
:101AB000E8CF01F1230E64EC0BF0E8CF02F1240E25
:101AC00064EC0BF0E8CF03F1010103AF96EF0DF0EA
:101AD00012EC32F0210E0C6E00C10BF04DEC0BF04D
:101AE000220E0C6E01C10BF04DEC0BF0230E0C6EB0
:101AF00002C10BF04DEC0BF0240E0C6E03C10BF089
:101B00004DEC0BF0210E64EC0BF0E8CF00F1220E4F
:101B100064EC0BF0E8CF01F1230E64EC0BF0E8CF9E
:101B200002F1240E64EC0BF0E8CF03F100C161F583
:101B300001C162F502C163F503C164F575EC34F0CF
:101B40005BEC33F0B3EC32F01590C70E64EC0BF0A5
:101B5000E8CF00F1010100B1B1EF0DF01592B2EF45
:101B60000DF0158281AAC0EF0DF015B4BBEF0DF09A
:101B70001580C0EF0DF070EC39F015A0D7EF39F0FB
:101B800007900001F28EF28C12AE03D012BC6EEF01
:101B900019F007B024EF2EF00FB014EF27F010BEAD
:101BA00014EF27F012B814EF27F000011650010AC5
:101BB000D8B41CEF1EF081BAE6EF0DF0000116500C
:101BC000040AD8B41AEF1CF0ECEF0DF00001165027
:101BD000040AD8B458EF1EF00301805181197F0B1D
:101BE000D8B424EF2EF013EE00F081517F0BE126E4
:101BF000812BE7CFE8FFE00BD8B424EF2EF023EEE3
:101C000082F0C2513F0BD926E7CFDFFFC22BDF5056
:101C1000780AD8A424EF2EF0078092C100F193C176
:101C200001F194C102F195C103F10101040E046FA9
:101C3000000E056F000E066F000E076FFDEC30F012
:101C400000AF2CEF0EF00101030E926F000E936FA8
:101C5000000E946F000E956F03018251720AD8B482
:101C600095EF26F08251520AD8B495EF26F08251B2
:101C7000750AD8B495EF26F08251680AD8B4AAEF55
:101C80000EF08251630AD8B4DEEF2AF08251690A5D
:101C9000D8B462EF21F082517A0AD8B475EF22F0FD
:101CA0008251490AD8B401EF21F08251500AD8B4C8
:101CB0001FEF20F08251700AD8B462EF20F08251F9
:101CC000540AD8B48DEF20F08251740AD8B4D3EFFF
:101CD00020F08251410AD8B4AFEF0FF082514B0A85
:101CE000D8B4ACEF0EF082516D0AD8B41FEF14F0E7
:101CF00082514D0AD8B438EF14F08251730AD8B427
:101D0000C5EF25F08251530AD8B42AEF26F082514C
:101D10004C0AD8B4C7EF14F08251590AD8B470EF06
:101D200013F012AE01D0128C15EF2BF0040114EE5B
:101D300000F080517F0BE12682C4E7FF802B120068
:101D400004010D0E826F96EC0EF00A0E826F96EC77
:101D50000EF0120013EF2BF004014B0E826F96EC85
:101D60000EF004012C0E826F96EC0EF081B802D0BA
:101D700036B630D003018351430AD8B4F1EF0EF0E8
:101D800003018351630AD8B4F3EF0EF003018351CA
:101D9000520AD8B4F5EF0EF003018351720AD8B499
:101DA000F7EF0EF003018351470AD8B4F9EF0EF0B4
:101DB00003018351670AD8B4FBEF0EF0030183518E
:101DC000540AD8B4FDEF0EF003018351740AD8B45D
:101DD0006DEF0FF003018351550AD8B4FFEF0EF0F9
:101DE00083D036807BD0369079D0368277D03692C9
:101DF00075D0368473D0369471D036866FD084C354
:101E000030F185C331F186C332F187C333F101016B
:101E1000296B60EC32F0D7EC31F000C104F101C164
:101E200005F102C106F103C107F153EC32F0200EB7
:101E3000F86EF76AF66A0900F5CF2CF10900F5CFC4
:101E40002DF10900F5CF2EF10900F5CF2FF1090092
:101E5000F5CF30F10900F5CF31F10900F5CF32F1BE
:101E60000900F5CF33F10101296B60EC32F0D7ECBA
:101E700031F0FDEC30F00101006746EF0FF0016733
:101E800046EF0FF0026746EF0FF0036701D025D051
:101E900004014E0E826F96EC0EF004016F0E826FFD
:101EA00096EC0EF004014D0E826F96EC0EF00401DC
:101EB000610E826F96EC0EF00401740E826F96EC48
:101EC0000EF00401630E826F96EC0EF00401680EB2
:101ED000826F96EC0EF013EF2BF03696CD0E0C6E53
:101EE00036C00BF04DEC0BF0CD0E64EC0BF0E8CFF0
:101EF00036F036B006D00401630E826F96EC0EF019
:101F000005D00401430E826F96EC0EF036B206D077
:101F10000401720E826F96EC0EF005D00401520E91
:101F2000826F96EC0EF036B406D00401670E826F15
:101F300096EC0EF005D00401470E826F96EC0EF081
:101F400036B606D00401740E826F96EC0EF005D002
:101F50000401540E826F96EC0EF013EF2BF0040187
:101F6000410E826F96EC0EF003018351310AD8B412
:101F700090EF12F003018351320AD8B4C0EF11F090
:101F800003018351330AD8B449EF11F0030183519F
:101F9000340AD8B439EF10F003018351350AD8B4AC
:101FA000D9EF0FF004013F0E826F96EC0EF013EFA5
:101FB0002BF003018451300AD8B4FFEF0FF0030176
:101FC0008451310AD8B402EF10F003018451650A3C
:101FD000D8B4F3EF0FF003018451640AD8B4F6EFDC
:101FE0000FF003EF10F03790F7EF0FF03780FB0E94
:101FF0000C6E37C00BF04DEC0BF003EF10F08B9034
:1020000003EF10F08B800401350E826F96EC0EF01A
:1020100004012C0E826F96EC0EF08BB017EF10F0CF
:102020000401300E826F96EC0EF01CEF10F00401EC
:10203000310E826F96EC0EF004012C0E826F96EC3E
:102040000EF0FB0E64EC0BF0E8CF37F037A030EF6A
:1020500010F00401640E826F96EC0EF035EF10F074
:102060000401650E826F96EC0EF037EF10F013EF5F
:102070002BF0CC0E64EC0BF0E8CF0BF004012C0E2F
:10208000826F96EC0EF003018451310AD8B45DEFF3
:1020900010F003018451300AD8B45FEF10F003014F
:1020A00084514D0AD8B469EF10F003018451540AE9
:1020B000D8B470EF10F087EF10F08A8401D08A94C2
:1020C0000BAE04D00BAC02D00BBA21D0E00E0B1239
:1020D00018D01F0E0B168539E844E00B0B1211D0F7
:1020E000E00E0B1653EC32F085C332F186C333F1A8
:1020F0000101296B60EC32F0D7EC31F000511F0B7D
:102100000B12CC0E0C6E0BC00BF04DEC0BF004015F
:10211000340E826F96EC0EF004012C0E826F96EC5A
:102120000EF0CC0E64EC0BF0E8CF1DF08AB406D0B4
:102130000401300E826F96EC0EF005D00401310ED2
:10214000826F96EC0EF004012C0E826F96EC0EF06E
:102150001D38E840070BE8CF82F40401300E8227D7
:1021600096EC0EF004012C0E826F96EC0EF012EC41
:1021700032F01D501F0BE8CF00F19BEC31F032C163
:1021800082F40401300E822796EC0EF033C182F403
:102190000401300E822796EC0EF004012C0E826FA3
:1021A00096EC0EF012EC32F030C000F100AF0BD024
:1021B000FF0E016FFF0E026FFF0E036F04012D0E65
:1021C000826F96EC0EF09BEC31F031C182F4040189
:1021D000300E822796EC0EF032C182F40401300EEC
:1021E000822796EC0EF033C182F40401300E822770
:1021F00096EC0EF004012C0E826F96EC0EF012ECB1
:1022000032F02FC000F19BEC31F031C182F40401B7
:10221000300E822796EC0EF032C182F40401300EAB
:10222000822796EC0EF033C182F40401300E82272F
:1022300096EC0EF004012C0E826F96EC0EF012EC70
:1022400032F031C000F100AF0BD0FF0E016FFF0E76
:10225000026FFF0E036F04012D0E826F96EC0EF0DD
:102260009BEC31F031C182F40401300E822796ECF0
:102270000EF032C182F40401300E822796EC0EF08B
:1022800033C182F40401300E822796EC0EF013EF76
:102290002BF0CB0E64EC0BF0E8CF0BF004012C0E0E
:1022A000826F96EC0EF003018451450AD8B46DEFAD
:1022B00011F003018451440AD8B470EF11F0030106
:1022C0008451300AD8B473EF11F003018451310AFC
:1022D000D8B477EF11F082EF11F00B9E7CEF11F084
:1022E0000B8E7CEF11F0FC0E0B167CEF11F0FC0E48
:1022F0000B160B807CEF11F0CB0E0C6E0BC00BF0AD
:102300004DEC0BF00401330E826F96EC0EF00401DD
:102310002C0E826F96EC0EF0CB0E64EC0BF0E8CF37
:102320001CF01CBE9BEF11F00401450E826F96EC71
:102330000EF0A0EF11F00401440E826F96EC0EF047
:1023400004012C0E826F96EC0EF00401300E826FA9
:1023500096EC0EF004012C0E826F96EC0EF01CB081
:10236000B9EF11F00401300E826F96EC0EF0BEEF63
:1023700011F00401310E826F96EC0EF013EF2BF08A
:10238000CA0E64EC0BF0E8CF0BF004012C0E826F48
:1023900096EC0EF003018451450AD8B4FCEF11F01D
:1023A00003018451440AD8B4FFEF11F003018451B2
:1023B0004D0AD8B408EF12F003018451410AD8B491
:1023C00002EF12F003018451460AD8B405EF12F06F
:1023D00003018451560AD8B410EF12F0030184515E
:1023E000500AD8B41BEF12F003018451520AD8B43A
:1023F0001EEF12F027EF12F00B9E21EF12F00B8E62
:1024000021EF12F00B9C21EF12F00B8C21EF12F058
:10241000FC0E0B1685C3E8FF030B0B1221EF12F025
:10242000C70E0B1685C3E8FF070BE846E846E846EB
:102430000B1221EF12F00B8421EF12F00B9421EF1D
:1024400012F0CA0E0C6E0BC00BF04DEC0BF0CA0E66
:1024500064EC0BF0E8CF1BF00401320E826F96ECB7
:102460000EF004012C0E826F96EC0EF01BBE40EFB6
:1024700012F00401450E826F96EC0EF045EF12F05B
:102480000401440E826F96EC0EF004012C0E826F54
:1024900096EC0EF01BC0E8FF030BE8CF82F40401BA
:1024A000300E822796EC0EF004012C0E826F96EC13
:1024B0000EF01BBC63EF12F00401410E826F96EC2C
:1024C0000EF068EF12F00401460E826F96EC0EF0EB
:1024D00004012C0E826F96EC0EF01BC0E8FF380B47
:1024E000E842E842E842E8CF82F40401300E822755
:1024F00096EC0EF004012C0E826F96EC0EF01BB4DD
:1025000089EF12F00401520E826F96EC0EF08EEFFE
:1025100012F00401500E826F96EC0EF013EF2BF0C8
:10252000C90E64EC0BF0E8CF0BF004012C0E826FA7
:1025300096EC0EF003018451450AD8B4AEEF12F0C8
:1025400003018451440AD8B4B1EF12F0030184515D
:102550004D0AD8B4B4EF12F0C2EF12F00B9EBCEFEC
:1025600012F00B8EBCEF12F0F80E0B1685C3E8FFCD
:10257000070B0B12BCEF12F0C90E0C6E0BC00BF068
:102580004DEC0BF00401310E826F96EC0EF004015D
:102590002C0E826F96EC0EF0C90E64EC0BF0E8CFB7
:1025A0001AF01ABE06D00401450E826F96EC0EF0AA
:1025B00005D00401440E826F96EC0EF004012C0E3F
:1025C000826F96EC0EF01AC0E8FF070BE8CF82F49A
:1025D0000401300E822796EC0EF004012C0E826F5F
:1025E00096EC0EF0078012EC32F02BC0E8FF003BB7
:1025F00000430043030B9BEC31F033C182F4040130
:10260000300E822796EC0EF004012C0E826F96ECB1
:102610000EF012EC32F02BC001F1019F019D2CC095
:1026200000F101019BEC31F02FC182F40401300E66
:10263000822796EC0EF030C182F40401300E82271E
:1026400096EC0EF031C182F40401300E822796EC34
:102650000EF032C182F40401300E822796EC0EF0A7
:1026600033C182F40401300E822796EC0EF004018F
:102670002C0E826F96EC0EF012EC32F02DC001F1B0
:102680002EC000F1D89001330033D89001330033CD
:1026900001019BEC31F02FC182F40401300E82273E
:1026A00096EC0EF030C182F40401300E822796ECD5
:1026B0000EF031C182F40401300E822796EC0EF048
:1026C00032C182F40401300E822796EC0EF033C141
:1026D00082F40401300E822796EC0EF013EF2BF0FB
:1026E000FC0E64EC0BF0E8CF0BF003018351520AAF
:1026F000D8B4A7EF13F003018351720AD8B4AAEF3C
:1027000013F003018351500AD8B4ADEF13F0030165
:102710008351700AD8B4B0EF13F003018351550A06
:10272000D8B4B3EF13F003018351750AD8B4B6EFF0
:1027300013F003018351430AD8B4BFEF13F0030130
:102740008351630AD8B4C2EF13F0CBEF13F00B90B0
:10275000C5EF13F00B80C5EF13F00B92C5EF13F02C
:102760000B82C5EF13F00B94C5EF13F00B84C5EF8C
:1027700013F00B96C5EF13F00B86C5EF13F00B9813
:10278000C5EF13F00B88C5EF13F0FC0E0C6E0BC0F9
:102790000BF04DEC0BF00401590E826F96EC0EF02D
:1027A0001190119211941198FC0E64EC0BF0E8CF8B
:1027B0000BF00BA011800BA211820BA411840BA8AB
:1027C000118811A0EBEF13F00401520E826F96EC0A
:1027D0000EF0F0EF13F00401720E826F96EC0EF023
:1027E00011A8FAEF13F00401430E826F96EC0EF07D
:1027F000FFEF13F00401630E826F96EC0EF011A24E
:1028000009EF14F00401500E826F96EC0EF00EEFFB
:1028100014F00401700E826F96EC0EF011A418EF04
:1028200014F00401550E826F96EC0EF01DEF14F0BB
:102830000401750E826F96EC0EF013EF2BF004017D
:102840006D0E826F96EC0EF003018351300AD8B4FE
:1028500077EF14F003018351310AD8B48AEF14F0F2
:1028600003018351320AD8B49DEF14F015EF2BF019
:1028700004014D0E826F96EC0EF053EC32F084C3DF
:1028800031F185C332F186C333F10101296B60EC6C
:1028900032F0D7EC31F003018351300AD8B45FEF46
:1028A00014F003018351310AD8B467EF14F0030127
:1028B0008351320AD8B46FEF14F015EF2BF0FD0EF0
:1028C0000C6E00C10BF04DEC0BF077EF14F0FE0E28
:1028D0000C6E00C10BF04DEC0BF08AEF14F0FF0E04
:1028E0000C6E00C10BF04DEC0BF09DEF14F00401E9
:1028F000300E826F96EC0EF004012C0E826F96EC77
:102900000EF012EC32F0FD0E64EC0BF0E8CF00F1AB
:10291000AEEF14F00401310E826F96EC0EF004015C
:102920002C0E826F96EC0EF012EC32F0FE0E64EC80
:102930000BF0E8CF00F1AEEF14F00401320E826F1D
:1029400096EC0EF012EC32F004012C0E826F96EC35
:102950000EF0FF0E64EC0BF0E8CF00F19BEC31F0D1
:1029600031C182F40401300E822796EC0EF032C1A0
:1029700082F40401300E822796EC0EF033C182F40B
:102980000401300E822796EC0EF013EF2BF00301BA
:102990008351300AD8B41BEF1AF003018351310A76
:1029A000D8B448EF1BF003018351320AD8B4B6EF14
:1029B0001BF003018351330AD8B4C6EF1BF00301A7
:1029C0008351340AD8B421EF1CF003018351350A36
:1029D000D8B470EF1EF003018351360AD8B49EEFCD
:1029E0001EF003018351370AD8B4F3EF17F0030147
:1029F0008351380AD8B491EF18F003018351440A87
:102A0000D8B41FEF16F003018351640AD8B43FEF26
:102A100016F003018351460AD8B475EF1DF0030187
:102A200083514D0AD8B46CEF16F0030183516D0A3F
:102A3000D8B486EF16F0030183515A0AD8B4C2EF16
:102A40001AF003018351490AD8B49EEF1FF0030125
:102A50008351500AD8B4D0EF1EF003018351540AB9
:102A6000D8B449EF1FF003018351630AD8B4A6EF2D
:102A700016F003018351430AD8B49EEF17F0030107
:102A80008351730AD8B4A4EF16F003018351610A8D
:102A9000D8B46CEF15F003018351650AD8B46BEF1D
:102AA0001AF003018351450AD8B479EF1AF00301F3
:102AB0008351620AD8B487EF1AF003018351420AA6
:102AC000D8B495EF1AF003018351760AD8B4A3EF76
:102AD0001AF0D8A415EF2BF004014C0E826F96EC7F
:102AE0000EF00401610E826F96EC0EF05BEC33F099
:102AF00004012C0E826F96EC0EF012EC32F0AFC592
:102B000000F101019BEC31F031C182F40401300E7F
:102B1000822796EC0EF032C182F40401300E822737
:102B200096EC0EF033C182F40401300E822796EC4D
:102B30000EF004012C0E826F96EC0EF012EC32F0C7
:102B4000B0C500F101019BEC31F031C182F4040108
:102B5000300E822796EC0EF032C182F40401300E62
:102B6000822796EC0EF033C182F40401300E8227E6
:102B700096EC0EF004012C0E826F96EC0EF012EC27
:102B800032F0B1C500F101019BEC31F031C182F4AA
:102B90000401300E822796EC0EF032C182F404015B
:102BA000300E822796EC0EF033C182F40401300E11
:102BB000822796EC0EF004012C0E826F96EC0EF03C
:102BC00012EC32F0B2C500F101019BEC31F031C1E1
:102BD00082F40401300E822796EC0EF032C182F4AA
:102BE0000401300E822796EC0EF033C182F404010A
:102BF000300E822796EC0EF004012C0E826F96ECBC
:102C00000EF012EC32F0B6C500F101019BEC31F090
:102C100031C182F40401300E822796EC0EF032C1ED
:102C200082F40401300E822796EC0EF033C182F458
:102C30000401300E822796EC0EF0CCEF1EF003015B
:102C40008451300AD8B42BEF16F003018451310AB5
:102C5000D8B42FEF16F01592159630EF16F01582B6
:102C6000C70E64EC0BF0E8CF00F10101008115A262
:102C70000091C70E0C6E00C10BF04DEC0BF0C70EAF
:102C800064EC0BF0E8CF00F1010100B14BEF16F05E
:102C900015924CEF16F0158204014C0E826F96ECE3
:102CA0000EF00401640E826F96EC0EF004012C0EFF
:102CB000826F96EC0EF015B265EF16F00401300E3F
:102CC000826F96EC0EF06AEF16F00401310E826FFF
:102CD00096EC0EF013EF2BF053EC32F084C333F18B
:102CE00060EC32F0D7EC31F0200E0C6E00C10BF02E
:102CF0004DEC0BF000C12FF505012F51000A06E045
:102D000005012F51010A02E0F5EC33F004014C0EED
:102D1000826F96EC0EF004014D0E826F96EC0EF071
:102D200004012C0E826F96EC0EF012EC32F02FC5DF
:102D300000F19BEC31F033C182F40401300E8227A4
:102D400096EC0EF0CCEF1EF0D7EF39F004014C0EEC
:102D5000826F96EC0EF00401630E826F96EC0EF01B
:102D6000B3EC32F004012C0E826F96EC0EF0BBEC4B
:102D700016F0CCEF1EF012EC32F0B5C500F10101F7
:102D8000003B0F0E00179BEC31F033C182F40401BD
:102D9000300E822796EC0EF0B5C500F101010F0E42
:102DA000010100179BEC31F033C182F40401300EB5
:102DB000822796EC0EF004012D0E826F96EC0EF039
:102DC000B4C500F10101003B0F0E00179BEC31F080
:102DD00033C182F40401300E822796EC0EF0B4C5A4
:102DE00000F101010F0E010100179BEC31F033C11E
:102DF00082F40401300E822796EC0EF004012D0EB1
:102E0000826F96EC0EF0B3C500F10101003B0F0E8E
:102E100000179BEC31F033C182F40401300E82279D
:102E200096EC0EF0B3C500F101010F0E0101001781
:102E30009BEC31F033C182F40401300E822796EC12
:102E40000EF00401200E826F96EC0EF0B2C500F178
:102E50000F0E010100179BEC31F033C182F4040125
:102E6000300E822796EC0EF00401200E826F96EC55
:102E70000EF0B1C500F101010101003B0F0E00177A
:102E80009BEC31F033C182F40401300E822796ECC2
:102E90000EF0B1C500F101010F0E010100179BEC0E
:102EA00031F033C182F40401300E822796EC0EF02B
:102EB00004013A0E826F96EC0EF0B0C500F10101EC
:102EC000003B0F0E00179BEC31F033C182F404017C
:102ED000300E822796EC0EF0B0C500F101010F0E06
:102EE000010100179BEC31F033C182F40401300E74
:102EF000822796EC0EF004013A0E826F96EC0EF0EB
:102F0000AFC500F10101003B0F0E00179BEC31F043
:102F100033C182F40401300E822796EC0EF0AFC567
:102F200000F101010F0E00179BEC31F033C182F468
:102F30000401300E822796EC0EF0120084C3E8FFE5
:102F40000F0BE83AE8CFB5F585C3E8FF0F0B050195
:102F5000B51387C3E8FF0F0BE83AE8CFB4F588C391
:102F6000E8FF0F0B0501B4138AC3E8FF0F0BE83A23
:102F7000E8CFB3F58BC3E8FF0F0B0501B3138DC387
:102F8000E8FF0F0BE8CFB2F58FC3E8FF0F0BE83A6D
:102F9000E8CFB1F590C3E8FF0F0B0501B11392C361
:102FA000E8FF0F0BE83AE8CFB0F593C3E8FF0F0B4B
:102FB0000501B01395C3E8FF0F0BE83AE8CFAFF572
:102FC00096C3E8FF0F0B0501AF130EEC33F00401BD
:102FD0004C0E826F96EC0EF00401430E826F96EC5D
:102FE0000EF0B0EF16F0078404014C0E826F96ECE1
:102FF0000EF00401370E826F96EC0EF004012C0ED9
:10300000826F96EC0EF005012E51130A06E00501C1
:103010002E51170A0DE08EEF18F00101000E006F1F
:10302000000E016F100E026F000E036F21EF18F0FB
:103030000101000E006F000E016F000E026F010E05
:10304000036F9BEC31F02AC182F40401300E822719
:1030500096EC0EF02BC182F40401300E822796EC20
:103060000EF02CC182F40401300E822796EC0EF093
:103070002DC182F40401300E822796EC0EF02EC191
:1030800082F40401300E822796EC0EF02FC182F4F8
:103090000401300E822796EC0EF030C182F4040158
:1030A000300E822796EC0EF031C182F40401300E0E
:1030B000822796EC0EF032C182F40401300E822792
:1030C00096EC0EF033C182F40401300E822796ECA8
:1030D0000EF004012C0E826F96EC0EF00101200E12
:1030E000006F000E016F000E026F000E036F9BEC6D
:1030F00031F031C182F40401300E822796EC0EF0DB
:1031000032C182F40401300E822796EC0EF033C1F6
:1031100082F40401300E822796EC0EF00794CCEF77
:103120001EF00501216B226B236B246B04014C0EF6
:10313000826F96EC0EF00401380E826F96EC0EF062
:1031400004012C0E826F96EC0EF00101200E006F30
:10315000000E016F000E026F000E036F9BEC31F04A
:103160002AC182F40401300E822796EC0EF02BC1A6
:1031700082F40401300E822796EC0EF02CC182F40A
:103180000401300E822796EC0EF02DC182F404016A
:10319000300E822796EC0EF02EC182F40401300E20
:1031A000822796EC0EF02FC182F40401300E8227A4
:1031B00096EC0EF030C182F40401300E822796ECBA
:1031C0000EF031C182F40401300E822796EC0EF02D
:1031D00032C182F40401300E822796EC0EF033C126
:1031E00082F40401300E822796EC0EF004012C0EBE
:1031F000826F96EC0EF025C500F126C501F127C5BA
:1032000002F128C503F10101200E046F000E056FC5
:10321000000E066F000E076F2EEC31F000C133F583
:1032200001C134F502C135F503C136F59BEC31F02F
:103230002AC182F40401300E822796EC0EF02BC1D5
:1032400082F40401300E822796EC0EF02CC182F439
:103250000401300E822796EC0EF02DC182F4040199
:10326000300E822796EC0EF02EC182F40401300E4F
:10327000822796EC0EF02FC182F40401300E8227D3
:1032800096EC0EF030C182F40401300E822796ECE9
:103290000EF031C182F40401300E822796EC0EF05C
:1032A00032C182F40401300E822796EC0EF033C155
:1032B00082F40401300E822796EC0EF0A0EC0EF0A2
:1032C000050133676BEF19F034676BEF19F0356761
:1032D0006BEF19F0366702D00AEF1AF0129E129CBB
:1032E00021C500F122C501F123C502F124C503F176
:1032F000899A400EC76E200EC66E9E96C69E0B0E15
:10330000C96EFF0E9EB602D0E82EFCD79E96C69ED2
:1033100002C1C9FFFF0E9EB602D0E82EFCD79E96D2
:10332000C69E01C1C9FFFF0E9EB602D0E82EFCD793
:103330009E96C69E00C1C9FFFF0E9EB602D0E82E23
:10334000FCD79E96C69EC952FF0E9EB602D0E82EAE
:10335000FCD70501200E326F040114EE00F08051FD
:103360007F0BE1269E96C69EC952FF0E9EB602D0E6
:10337000E82EFCD7C9CFE7FF0401802B0501322FCF
:10338000ACEF19F0898A33C500F134C501F135C5B8
:1033900002F136C503F10101010E046F000E056F45
:1033A000000E066F000E076FFDEC30F000C133F524
:1033B00001C134F502C135F503C136F505013367A6
:1033C000E9EF19F03467E9EF19F03567E9EF19F023
:1033D000366702D00AEF1AF021C500F122C501F1CB
:1033E00023C502F124C503F10101200E046F000E74
:1033F000056F000E066F000E076F02EC31F000C182
:1034000021F501C122F502C123F503C124F5128E75
:1034100015EF2BF00401450E826F96EC0EF00401BF
:103420004F0E826F96EC0EF00401460E826F96EC02
:103430000EF0CCEF1EF0078431EC39F012EC32F0D4
:103440002DC500F19BEC31F004014C0E826F96EC1F
:103450000EF00401300E826F96EC0EF004012C0E7B
:10346000826F96EC0EF031C182F40401300E822797
:1034700096EC0EF032C182F40401300E822796ECF5
:103480000EF033C182F40401300E822796EC0EF068
:1034900004012C0E826F96EC0EF012EC32F02EC569
:1034A00000F19BEC31F031C182F40401300E82272F
:1034B00096EC0EF032C182F40401300E822796ECB5
:1034C0000EF033C182F40401300E822796EC0EF028
:1034D0000794CCEF1EF004014C0E826F96EC0EF0B8
:1034E0000401650E826F96EC0EF0D1EC34F0CCEF57
:1034F0001EF004014C0E826F96EC0EF00401450E96
:10350000826F96EC0EF0E8EC34F0CCEF1EF0040184
:103510004C0E826F96EC0EF00401620E826F96ECF8
:103520000EF016EC35F0CCEF1EF004014C0E826F5D
:1035300096EC0EF00401420E826F96EC0EF0FFEC5A
:1035400034F0CCEF1EF004014C0E826F96EC0EF0BE
:103550000401760E826F96EC0EF004012C0E826F41
:1035600096EC0EF010A807D00401310E826F96EC95
:103570000EF0CCEF1EF00401300E826F96EC0EF0D0
:10358000CCEF1EF004014C0E826F96EC0EF004019D
:103590005A0E826F96EC0EF004012C0E826F96ECA0
:1035A0000EF031EC39F012EC32F005012E51130A15
:1035B00006E005012E51170A0DE0F3EF1AF00101A4
:1035C000000E006F000E016F100E026F000E036FF1
:1035D000F3EF1AF00101000E006F000E016F000EF4
:1035E000026F010E036F0101200E046F000E056FC4
:1035F000000E066F000E076F2EEC31F09BEC31F0E1
:103600002AC182F40401300E822796EC0EF02BC101
:1036100082F40401300E822796EC0EF02CC182F465
:103620000401300E822796EC0EF02DC182F40401C5
:10363000300E822796EC0EF02EC182F40401300E7B
:10364000822796EC0EF02FC182F40401300E8227FF
:1036500096EC0EF030C182F40401300E822796EC15
:103660000EF031C182F40401300E822796EC0EF088
:1036700032C182F40401300E822796EC0EF033C181
:1036800082F40401300E822796EC0EF0CCEF1EF08F
:10369000078404014C0E826F96EC0EF00401310E8B
:1036A000826F96EC0EF004012C0E826F96EC0EF0F9
:1036B00025C500F126C501F127C502F128C503F192
:1036C0000101200E046F000E056F000E066F000E44
:1036D000076F2EEC31F09BEC31F02AC182F404012B
:1036E000300E822796EC0EF02BC182F40401300ECE
:1036F000822796EC0EF02CC182F40401300E822752
:1037000096EC0EF02DC182F40401300E822796EC67
:103710000EF02EC182F40401300E822796EC0EF0DA
:103720002FC182F40401300E822796EC0EF030C1D6
:1037300082F40401300E822796EC0EF031C182F43F
:103740000401300E822796EC0EF032C182F404019F
:10375000300E822796EC0EF033C182F40401300E55
:10376000822796EC0EF00794CCEF1EF0078404013C
:103770004C0E826F96EC0EF00401320E826F96ECC6
:103780000EF005EC37F00794CCEF1EF0078437B04D
:10379000CCEF1BF0DFEF1BF0010E166E04014C0E98
:1037A000826F96EC0EF00401330E826F96EC0EF0F1
:1037B00062EC37F0000E166E079453EF1BF0020E0A
:1037C000166E62EC37F08B800501010E306F3C0EF7
:1037D000316F01015E6B5F6B606B616B626B636B82
:1037E000646B656B666B676B686B696B536B546B73
:1037F000CF6ACE6A0F9A0F9C0F9E030E166E0401BD
:103800004C0E826F96EC0EF00401330E826F96EC34
:103810000EF004012C0E826F96EC0EF004012D0EBA
:10382000826F96EC0EF00401310E826F96EC0EF072
:1038300013EF2BF062EC37F0000E166E8B9015EF45
:103840002BF0078404014C0E826F96EC0EF00401FD
:10385000340E826F96EC0EF004012C0E826F96EC03
:103860000EF053EC32F084C32AF185C32BF186C3EA
:103870002CF187C32DF188C32EF189C32FF18AC3A0
:1038800030F18BC331F18CC332F18DC333F10101BF
:10389000296B60EC32F0D7EC31F0200E046F000E93
:1038A000056F000E066F000E076F0EEC31F000C1C1
:1038B00021F501C122F502C123F503C124F5E4EC91
:1038C00038F038C5AFF539C5B0F53AC5B1F53BC5E7
:1038D000B2F53CC5B3F53DC5B4F53EC5B5F5BBEC99
:1038E00016F004012C0E826F96EC0EF03FC500F12D
:1038F00040C501F141C502F142C503F10101000ECD
:10390000046F000E056F010E066F000E076F2EECA0
:1039100031F09BEC31F0296790EF1CF095EF1CF033
:1039200004012D0E826F96EC0EF030C182F404017A
:10393000300E822796EC0EF031C182F40401300E75
:10394000822796EC0EF004012E0E826F96EC0EF09C
:1039500032C182F40401300E822796EC0EF033C19E
:1039600082F40401300E822796EC0EF004012C0E36
:10397000826F96EC0EF012EC32F043C500F144C5B4
:1039800001F13FEC2CF004012C0E826F96EC0EF04E
:1039900012EC32F045C500F19BEC31F031C182F4FC
:1039A0000401300E822796EC0EF032C182F404013D
:1039B000300E822796EC0EF033C182F40401300EF3
:1039C000822796EC0EF004012C0E826F96EC0EF01E
:1039D00037C5E8FFE8B806D00401300E826F96ECD8
:1039E0000EF005D00401310E826F96EC0EF004014A
:1039F0002C0E826F96EC0EF037C5E8FFE8BA06D0C1
:103A00000401300E826F96EC0EF06CD00401310E82
:103A1000826F96EC0EF004012C0E826F96EC0EF085
:103A200047C500F148C501F149C502F14AC503F196
:103A3000BDEC31F05EEC2FF004012C0E826F96ECA1
:103A40000EF04BC500F14CC501F14DC502F14EC55C
:103A500003F10101000E046F000E056F010E066FE9
:103A6000000E076F2EEC31F09BEC31F029673BEF35
:103A70001DF040EF1DF004012D0E826F96EC0EF04C
:103A800030C182F40401300E822796EC0EF031C171
:103A900082F40401300E822796EC0EF004012E0E03
:103AA000826F96EC0EF032C182F40401300E822750
:103AB00096EC0EF033C182F40401300E822796ECAE
:103AC0000EF004012C0E826F96EC0EF04FC500F143
:103AD00050C501F151C502F152C503F1BDEC31F001
:103AE0005EEC2FF00794CCEF1EF053EC32F085C360
:103AF0002AF186C32BF187C32CF188C32DF189C32A
:103B00002EF18AC32FF18BC330F18CC331F18DC3F9
:103B100032F18EC333F10101296B60EC32F0D7EC46
:103B200031F00101010E046F000E056F000E066FEB
:103B3000000E076FFDEC30F0100E046F000E056FE5
:103B4000000E066F000E076F0EEC31F000C129F574
:103B500001C12AF502C12BF503C12CF58CEC36F01E
:103B600004014C0E826F96EC0EF00401460E826F3B
:103B700096EC0EF004012C0E826F96EC0EF025C52B
:103B800000F126C501F127C502F128C503F10101A5
:103B9000100E046F000E056F000E066F000E076F0B
:103BA0002EEC31F09BEC31F02AC182F40401300E8E
:103BB000822796EC0EF02BC182F40401300E82278E
:103BC00096EC0EF02CC182F40401300E822796ECA4
:103BD0000EF02DC182F40401300E822796EC0EF017
:103BE0002EC182F40401300E822796EC0EF02FC114
:103BF00082F40401300E822796EC0EF030C182F47C
:103C00000401300E822796EC0EF031C182F40401DB
:103C1000300E822796EC0EF032C182F40401300E91
:103C2000822796EC0EF033C182F40401300E822715
:103C300096EC0EF0CCEF1EF037B021EF1EF0020E26
:103C4000166E62EC37F000011650020AD8B43FEF4E
:103C50001EF005012F51010AD8B435EF1EF015B240
:103C60003AEF1EF081BA3AEF1EF0000E166E158480
:103C700015EF2BF0050E166E1584D7EF39F08B80FB
:103C800001015E6B5F6B606B616B626B636B646B9E
:103C9000656B666B676B686B696B536B546BCF6A54
:103CA000CE6A0F9A0F9C0F9E030E166E15EF2BF027
:103CB00062EC37F005012F51010AD8B466EF1EF00F
:103CC00015B26BEF1EF081BA6BEF1EF0000E166E90
:103CD000158415EF2BF0050E166E1584D7EF39F00D
:103CE00004014C0E826F96EC0EF00401350E826FCB
:103CF00096EC0EF004012C0E826F96EC0EF012EC96
:103D000032F00784B9C500F107949BEC31F031C162
:103D100082F40401300E822796EC0EF032C182F458
:103D20000401300E822796EC0EF033C182F40401B8
:103D3000300E822796EC0EF0CCEF1EF025EC37F01B
:103D400012EC32F037C500F19BEC31F004014C0E5F
:103D5000826F96EC0EF00401360E826F96EC0EF038
:103D600004012C0E826F96EC0EF031C182F4040136
:103D7000300E822796EC0EF032C182F40401300E30
:103D8000822796EC0EF033C182F40401300E8227B4
:103D900096EC0EF0CCEF1EF0A0EC0EF015EF2BF031
:103DA00004014C0E826F96EC0EF00401500E826FEF
:103DB00096EC0EF004012C0E826F96EC0EF085C38B
:103DC0002AF186C32BF187C32CF188C32DF189C357
:103DD0002EF18AC32FF18BC330F18CC331F18DC327
:103DE00032F18EC333F1010160EC32F0D7EC31F0E7
:103DF00003018451530A0DE0030184514D0A38E058
:103E00000401780E826F96EC0EF0A0EC0EF015EF28
:103E10002BF00401530E826F96EC0EF0250E0C6E03
:103E200000C10BF04DEC0BF0260E0C6E01C10BF037
:103E30004DEC0BF0270E0C6E02C10BF04DEC0BF0AD
:103E4000280E0C6E03C10BF04DEC0BF000C157F5C2
:103E500001C158F502C159F503C15AF500C15BF51E
:103E600001C15CF502C15DF503C15EF5ADEF1FF068
:103E700004014D0E826F96EC0EF0290E0C6E00C1FF
:103E80000BF04DEC0BF000C15FF500C160F5ADEF3C
:103E90001FF004014C0E826F96EC0EF00401540EDC
:103EA000826F96EC0EF004012C0E826F96EC0EF0F1
:103EB00084C32AF185C32BF186C32CF187C32DF16E
:103EC00088C32EF189C32FF18AC330F18BC331F13E
:103ED0008DC332F18EC333F1010160EC32F0D7ECC7
:103EE00031F00101000E046F000E056F010E066F28
:103EF000000E076F0EEC31F0210E0C6E00C10BF0BE
:103F00004DEC0BF0220E0C6E01C10BF04DEC0BF0E2
:103F1000230E0C6E02C10BF04DEC0BF0240E0C6E58
:103F200003C10BF04DEC0BF000C161F501C162F56E
:103F300002C163F503C164F5ADEF1FF004014C0E3F
:103F4000826F96EC0EF00401490E826F96EC0EF033
:103F500004012C0E826F96EC0EF0250E64EC0BF033
:103F6000E8CF00F1260E64EC0BF0E8CF01F1270E4C
:103F700064EC0BF0E8CF02F1280E64EC0BF0E8CF14
:103F800003F19BEC31F05EEC2FF00401730E826FB5
:103F900096EC0EF004012C0E826F96EC0EF012ECF3
:103FA00032F0290E64EC0BF0E8CF00F19BEC31F01D
:103FB0005EEC2FF004016D0E826F96EC0EF00401A2
:103FC0002C0E826F96EC0EF05BC500F15CC501F122
:103FD0005DC502F15EC503F19BEC31F05EEC2FF0A4
:103FE0000401730E826F96EC0EF004012C0E826FAA
:103FF00096EC0EF012EC32F060C500F19BEC31F063
:104000005EEC2FF004016D0E826F96EC0EF0040151
:104010002C0E826F96EC0EF061C500F162C501F1C5
:1040200063C502F164C503F130EC2BF004012C0EE2
:10403000826F96EC0EF0A0EC0EF015EF2BF083C320
:104040002AF184C32BF185C32CF186C32DF187C3DC
:104050002EF188C32FF189C330F18AC331F18BC3AC
:1040600032F18CC333F1010160EC32F0D7EC31F066
:10407000160E0C6E00C10BF04DEC0BF0170E0C6E13
:1040800001C10BF04DEC0BF0180E0C6E02C10BF0E1
:104090004DEC0BF0190E0C6E03C10BF04DEC0BF058
:1040A00000C18EF101C18FF102C190F103C191F104
:1040B00000C192F101C193F102C194F103C195F1E4
:1040C00001EF21F083C32AF184C32BF185C32CF1C6
:1040D00086C32DF187C32EF188C32FF189C330F138
:1040E0008AC331F18BC332F18CC333F1010160EC2F
:1040F00032F0D7EC31F000C18EF101C18FF102C175
:1041000090F103C191F100C192F101C193F102C19B
:1041100094F103C195F101EF21F083C32AF184C327
:104120002BF185C32CF186C32DF187C32EF188C3F3
:104130002FF189C330F18AC331F18CC332F18DC3C1
:1041400033F1010160EC32F0D7EC31F00101000EE7
:10415000046F000E056F010E066F000E076F0EEC68
:1041600031F01A0E0C6E00C10BF04DEC0BF01B0E73
:104170000C6E01C10BF04DEC0BF01C0E0C6E02C16D
:104180000BF04DEC0BF01D0E0C6E03C10BF04DEC63
:104190000BF000C196F101C197F102C198F103C182
:1041A00099F101EF21F083C32AF184C32BF185C378
:1041B0002CF186C32DF187C32EF188C32FF189C35B
:1041C00030F18AC331F18CC332F18DC333F1010177
:1041D00060EC32F0D7EC31F00101000E046F000EFC
:1041E000056F010E066F000E076F0EEC31F000C177
:1041F00096F101C197F102C198F103C199F101EF64
:1042000021F0160E64EC0BF0E8CF00F1170E64EC11
:104210000BF0E8CF01F1180E64EC0BF0E8CF02F1DF
:10422000190E64EC0BF0E8CF03F19BEC31F05EEC7F
:104230002FF00401730E826F96EC0EF004012C0E29
:10424000826F96EC0EF08EC100F18FC101F190C12A
:1042500002F191C103F19BEC31F05EEC2FF004010F
:10426000730E826F96EC0EF004012C0E826F96ECAA
:104270000EF01A0E64EC0BF0E8CF00F11B0E64ECAC
:104280000BF0E8CF01F11C0E64EC0BF0E8CF02F16B
:104290001D0E64EC0BF0E8CF03F130EC2BF00401C1
:1042A0002C0E826F96EC0EF096C100F197C101F1D1
:1042B00098C102F199C103F130EC2BF0A0EC0EF0A3
:1042C00015EF2BF00401690E826F96EC0EF00401DD
:1042D0002C0E826F96EC0EF00101040E006F000EA2
:1042E000016F000E026F000E036F9BEC31F02CC1CA
:1042F00082F40401300E822796EC0EF02DC182F478
:104300000401300E822796EC0EF02EC182F40401D7
:10431000300E822796EC0EF02FC182F40401300E8D
:10432000822796EC0EF030C182F40401300E822711
:1043300096EC0EF031C182F40401300E822796EC27
:104340000EF032C182F40401300E822796EC0EF09A
:1043500033C182F40401300E822796EC0EF0040182
:104360002C0E826F96EC0EF001010D0E006F000E08
:10437000016F000E026F000E036F9BEC31F02CC139
:1043800082F40401300E822796EC0EF02DC182F4E7
:104390000401300E822796EC0EF02EC182F4040147
:1043A000300E822796EC0EF02FC182F40401300EFD
:1043B000822796EC0EF030C182F40401300E822781
:1043C00096EC0EF031C182F40401300E822796EC97
:1043D0000EF032C182F40401300E822796EC0EF00A
:1043E00033C182F40401300E822796EC0EF00401F2
:1043F0002C0E826F96EC0EF001014C0E006F000E39
:10440000016F000E026F000E036F9BEC31F02CC1A8
:1044100082F40401300E822796EC0EF02DC182F456
:104420000401300E822796EC0EF02EC182F40401B6
:10443000300E822796EC0EF02FC182F40401300E6C
:10444000822796EC0EF030C182F40401300E8227F0
:1044500096EC0EF031C182F40401300E822796EC06
:104460000EF032C182F40401300E822796EC0EF079
:1044700033C182F40401300E822796EC0EF0040161
:104480002C0E826F96EC0EF0200EF86EF76AF66A2C
:1044900004010900F5CF82F496EC0EF00900F5CF87
:1044A00082F496EC0EF00900F5CF82F496EC0EF053
:1044B0000900F5CF82F496EC0EF00900F5CF82F4F6
:1044C00096EC0EF00900F5CF82F496EC0EF00900A0
:1044D000F5CF82F496EC0EF00900F5CF82F496EC5D
:1044E0000EF0A0EC0EF015EF2BF08351630AD8A468
:1044F00013EF2BF08451610AD8A413EF2BF08551F0
:104500006C0AD8A413EF2BF08651410A3FE0865184
:10451000440A1BE08651420AD8B4D9EF22F08651F2
:10452000350AD8B49FEF2CF08651360AD8B4F4EF90
:104530002CF08651370AD8B45DEF2DF08651380A39
:10454000D8B4BBEF2DF013EF2BF00798079A0401B6
:104550007A0E826F96EC0EF00401780E826F96EC64
:104560000EF00401640E826F96EC0EF00401550EFD
:10457000826F96EC0EF0C2EF22F004014C0E826FB7
:1045800096EC0EF0A0EC0EF015EF2BF00788079AD2
:1045900004017A0E826F96EC0EF00401410E826FD8
:1045A00096EC0EF00401610E826F96EC0EF0B6EF01
:1045B00022F00798078A04017A0E826F96EC0EF0BB
:1045C0000401420E826F96EC0EF00401610E826FC0
:1045D00096EC0EF0B6EF22F001016667F7EF22F0DD
:1045E0006767F7EF22F06867F7EF22F0696716D088
:1045F00001014F6703EF23F0506703EF23F051678A
:1046000003EF23F052670AD00101000E006F000E85
:10461000016F000E026F000E036F120011B80AD076
:104620000101620E046F010E056F000E066F000E91
:10463000076F09D00101A70E046F020E056F000E6F
:10464000066F000E076F66C100F167C101F168C116
:1046500002F169C103F1FDEC30F003BFA0EF23F0DC
:10466000119A119C0101000E046FA80E056F550EE2
:10467000066F020E076F66C100F167C101F168C1E4
:1046800002F169C103F166C18AF167C18BF168C1AA
:104690008CF169C18DF1FDEC30F003BF0BD001014D
:1046A000000E8A6FA80E8B6F550E8C6F020E8D6FE9
:1046B000118A119C0E0E64EC0BF0E8CF18F10F0E6E
:1046C00064EC0BF0E8CF19F1100E64EC0BF0E8CFBE
:1046D0001AF1110E64EC0BF0E8CF1BF146EC30F050
:1046E0008AC104F18BC105F18CC106F18DC107F1BE
:1046F000FDEC30F007820AEC30F046EC30F0079227
:104700000AEC30F08AC100F18BC101F18CC102F1D9
:104710008DC103F107920AEC30F0CC0E046FE00E6D
:10472000056F870E066F050E076FFDEC30F000C1B8
:1047300018F101C119F102C11AF103C11BF140D0F6
:1047400013AAA5EF23F0138E139A119C119A01015D
:10475000800E006F1A0E016F060E026F000E036FBF
:104760004FC104F150C105F151C106F152C107F129
:10477000FDEC30F003AF05D012EC32F0118C119A41
:1047800012000E0E64EC0BF0E8CF18F10F0E64EC83
:104790000BF0E8CF19F1100E64EC0BF0E8CF1AF132
:1047A000110E64EC0BF0E8CF1BF14FC100F150C1CA
:1047B00001F151C102F152C103F107820AEC30F05C
:1047C00018C100F119C101F11AC102F11BC103F1B5
:1047D00012000784BAC166F1BBC167F1BCC168F1C0
:1047E000BDC169F14BC14FF14CC150F14DC151F107
:1047F0004EC152F157C159F158C15AF10794010104
:1048000066670AEF24F067670AEF24F068670AEF2B
:1048100024F0696716D001014F6716EF24F0506746
:1048200016EF24F0516716EF24F052670AD0010109
:10483000000E006F000E016F000E026F000E036F7E
:10484000120011B80AD00101620E046F010E056F4B
:10485000000E066F000E076F09D00101A70E046F4E
:10486000020E056F000E066F000E076F66C100F1A5
:1048700067C101F168C102F169C103F1FDEC30F0DB
:1048800003BFA2EF24F00101000E046FA80E056F14
:10489000550E066F020E076F66C100F167C101F188
:1048A00068C102F169C103F166C18AF167C18BF188
:1048B00068C18CF169C18DF1FDEC30F003BF09D006
:1048C0000101000E8A6FA80E8B6F550E8C6F020EC1
:1048D0008D6F46EC30F000C104F101C105F102C159
:1048E00006F103C107F1000E006FA00E016F980ED4
:1048F000026F7B0E036F2EEC31F000C118F101C185
:1049000019F102C11AF103C11BF1000E006FA00ED4
:10491000016F980E026F7B0E036F8AC104F18BC189
:1049200005F18CC106F18DC107F12EEC31F018C1F3
:1049300004F119C105F11AC106F11BC107F1FDEC23
:1049400030F012000101A80E006F610E016F000E21
:10495000026F000E036F4FC104F150C105F151C148
:1049600006F152C107F1FDEC30F003AF0AD00101AE
:10497000A80E006F610E016F000E026F000E036F34
:1049800000D0C80E006FAF0E016F000E026F000E58
:10499000036F4FC104F150C105F151C106F152C17D
:1049A00007F10EEC31F012000784BAC166F1BBC109
:1049B00067F1BCC168F1BDC169F14BC14FF14CC198
:1049C00050F14DC151F14EC152F157C159F158C189
:1049D0005AF1079401016667F5EF24F06767F5EF78
:1049E00024F06867F5EF24F0696716D001014F677E
:1049F00001EF25F0506701EF25F0516701EF25F039
:104A000052670AD00101000E006F000E016F000E08
:104A1000026F000E036F120011B80AD00101620E7E
:104A2000046F010E056F000E066F000E076F09D0B0
:104A30000101A70E046F020E056F000E066F000E37
:104A4000076F66C100F167C101F168C102F169C178
:104A500003F1FDEC30F003BFB7EF25F00101000ECC
:104A6000046FA80E056F550E066F020E076F66C124
:104A700000F167C101F168C102F169C103F166C1CA
:104A80008AF167C18BF168C18CF169C18DF1FDECD0
:104A900030F003BF09D00101000E8A6FA80E8B6FA2
:104AA000550E8C6F020E8D6F010E006F000E016FA0
:104AB000000E026F000E036F8AC104F18BC105F175
:104AC0008CC106F18DC107F12EEC31F018C104F153
:104AD00019C105F11AC106F11BC107F19BEC31F0B8
:104AE0002AC182F40401300E822796EC0EF02BC10D
:104AF00082F40401300E822796EC0EF02CC182F471
:104B00000401300E822796EC0EF02DC182F40401D0
:104B1000300E822796EC0EF02EC182F40401300E86
:104B2000822796EC0EF02FC182F40401300E82270A
:104B300096EC0EF030C182F40401300E822796EC20
:104B40000EF031C182F40401300E822796EC0EF093
:104B500032C182F40401300E822796EC0EF033C18C
:104B600082F40401300E822796EC0EF012004FC141
:104B700000F150C101F151C102F152C103F1010133
:104B80009BEC31F05EEC2FF012000401730E826F8B
:104B900096EC0EF004012C0E826F96EC0EF007845A
:104BA00062C166F163C167F164C168F165C169F111
:104BB0004BC14FF14CC150F14DC151F14EC152F1B9
:104BC00057C159F158C15AF10794EBEC25F0A0EC0C
:104BD0000EF015EF2BF066C100F167C101F168C15D
:104BE00002F169C103F101019BEC31F05EEC2FF0A1
:104BF0000401630E826F96EC0EF004012C0E826F9E
:104C000096EC0EF04FC100F150C101F151C102F11B
:104C100052C103F101019BEC31F05EEC2FF0040175
:104C2000660E826F96EC0EF004012C0E826F96ECED
:104C30000EF012EC32F059C100F15AC101F101013C
:104C40009BEC31F05EEC2FF00401740E826F96EC59
:104C50000EF0120010820401530E826F96EC0EF0DB
:104C600004012C0E826F96EC0EF083C32AF184C3EC
:104C70002BF185C32CF186C32DF187C32EF188C398
:104C80002FF189C330F18AC331F18BC332F18CC368
:104C900033F1010160EC32F0D7EC31F000C166F184
:104CA00001C167F102C168F103C169F18EC32AF144
:104CB0008FC32BF190C32CF191C32DF192C32EF130
:104CC00093C32FF194C330F195C331F196C332F100
:104CD00097C333F1010160EC32F0D7EC31F000C141
:104CE0004FF101C150F102C151F103C152F153EC36
:104CF00032F099C32FF19AC330F19BC331F19CC3B9
:104D000032F19DC333F1010160EC32F0D7EC31F0A8
:104D100000C159F101C15AF1EBEC25F004012C0E50
:104D2000826F96EC0EF0A5EF26F0118E1CA002D03B
:104D30001CAE108C1BBE02D01BA4108E030182512E
:104D4000520A02E10F8201D00F928251750A02E1EC
:104D5000108401D010948251550A02E1108601D0CE
:104D600010968351310A03E11382138402D0139207
:104D7000139403018351660A01E056D00401660EC4
:104D8000826F96EC0EF004012C0E826F96EC0EF002
:104D9000E9EC23F09BEC31F02AC182F40401300EDF
:104DA000822796EC0EF02BC182F40401300E82278C
:104DB00096EC0EF02CC182F40401300E822796ECA2
:104DC0000EF02DC182F40401300E822796EC0EF015
:104DD0002EC182F40401300E822796EC0EF02FC112
:104DE00082F40401300E822796EC0EF030C182F47A
:104DF0000401300E822796EC0EF031C182F40401DA
:104E0000300E822796EC0EF032C182F40401300E8F
:104E1000822796EC0EF033C182F40401300E822713
:104E200096EC0EF013EF2BF011A003D011A401D0DB
:104E30001084078410B27EEF27F010A462EF27F0F1
:104E4000BAC166F1BBC167F1BCC168F1BDC169F10E
:104E5000BEC16AF1BFC16BF1C0C16CF1C1C16DF1DE
:104E6000C2C16EF1C3C16FF1C4C170F1C5C171F1AE
:104E7000C6C172F1C7C173F1C8C174F1C9C175F17E
:104E8000CAC176F1CBC177F1CCC178F1CDC179F14E
:104E9000CEC17AF1CFC17BF1D0C17CF1D1C17DF11E
:104EA000D2C17EF1D3C17FF1D4C180F1D5C181F1EE
:104EB000D6C182F1D7C183F1D8C184F1D9C185F1BE
:104EC0006AEF27F062C166F163C167F164C168F1FE
:104ED00065C169F1BAC186F1BBC187F1BCC188F176
:104EE000BDC189F14BC14FF14CC150F14DC151F1E0
:104EF0004EC152F157C159F158C15AF107940FA050
:104F0000A0EF27F0010196678DEF27F097678DEFEF
:104F100027F098678DEF27F0996791EF27F0A0EFC2
:104F200027F0ECEC22F096C104F197C105F198C18D
:104F300006F199C107F1FDEC30F003BFD9EF2AF07B
:104F4000ECEC22F00101000E046F000E056F010E63
:104F5000066F000E076F2EEC31F011A02AD011A2BF
:104F600028D09BEC31F0296701D005D004012D0E2B
:104F7000826F96EC0EF030C182F40401300E82276D
:104F800096EC0EF031C182F40401300E822796ECCB
:104F90000EF032C182F40401300E822796EC0EF03E
:104FA00033C182F40401300E822796EC0EF0A0EC9F
:104FB0000EF012A8C5D012981DC01EF01E3A1E4257
:104FC000070E1E1600011E50000AD8B46CEF28F020
:104FD00000011E50010AD8B4F8EF27F000011E505E
:104FE000020AD8B4F6EF27F09EEF28F09EEF28F0E3
:104FF00012EC32F02DC001F12EC000F1D890013337
:105000000033D890013300330101630E046F000EAA
:10501000056F000E066F000E076F2EEC31F0280EA4
:10502000046F000E056F000E066F000E076FFDEC9B
:1050300030F000C130F012EC32F02BC001F1019FD2
:10504000019D2CC000F10101A40E046F000E056F3C
:10505000000E066F000E076F2EEC31F000C12FF02E
:1050600000C104F101C105F102C106F103C107F15C
:10507000640E006F000E016F000E026F000E036FD2
:10508000FDEC30F0050E046F000E056F000E066F8C
:10509000000E076F2EEC31F000C104F101C105F1E3
:1050A00002C106F103C107F112EC32F030C000F189
:1050B000FDEC30F000C131F031C0E8FF050F305C8D
:1050C00003E78A849EEF28F031C0E8FF0A0F305CC6
:1050D00001E68A949EEF28F000C124F101C125F178
:1050E00002C126F103C127F112EC32F018EC32F0C4
:1050F0001D501F0BE8CF00F10101640E046F000E7C
:10510000056F000E066F000E076F0EEC31F024C124
:1051100004F125C105F126C106F127C107F1FDEC17
:1051200030F003BF02D08A9401D08A8424C100F1F8
:1051300025C101F126C102F127C103F115EF2BF0C2
:1051400000C124F101C125F102C126F103C127F1FB
:1051500010AE4DD0109E00C108F101C109F102C18D
:105160000AF103C10BF19BEC31F030C1E2F131C126
:10517000E3F132C1E4F133C1E5F108C100F109C145
:1051800001F10AC102F10BC103F101016C0E046FC0
:10519000070E056F000E066F000E076FFDEC30F076
:1051A00003BF04D00101550EE66F1CD008C100F109
:1051B00009C101F10AC102F10BC103F10101A40E01
:1051C000046F060E056F000E066F000E076FFDECF4
:1051D00030F003BF04D001017F0EE66F03D0010160
:1051E000FF0EE66F1F8E11AED9EF2AF0119E24C17B
:1051F00000F125C101F126C102F127C103F111A07F
:1052000005D011A203D00FB0D9EF2AF010A410EFEF
:1052100029F00401750E826F96EC0EF015EF29F05F
:105220000401720E826F96EC0EF004012C0E826F58
:1052300096EC0EF09BEC31F0296724EF29F0040185
:10524000200E826F27EF29F004012D0E826F96EC5D
:105250000EF030C182F40401300E822796EC0EF07D
:1052600031C182F40401300E822796EC0EF0040165
:105270002E0E826F96EC0EF032C182F40401300ED5
:10528000822796EC0EF033C182F40401300E82279F
:1052900096EC0EF004016D0E826F96EC0EF0040198
:1052A0002C0E826F96EC0EF04FC100F150C101F14F
:1052B00051C102F152C103F101019BEC31F05EECEE
:1052C0002FF00401480E826F96EC0EF004017A0E66
:1052D000826F96EC0EF004012C0E826F96EC0EF0AD
:1052E00066C100F167C101F168C102F169C103F152
:1052F00001019BEC31F05EEC2FF00401630E826F34
:1053000096EC0EF004012C0E826F96EC0EF066C146
:1053100000F167C101F168C102F169C103F1010146
:105320000A0E046F000E056F000E066F000E076F69
:105330000EEC31F0000E046F120E056F000E066FBA
:10534000000E076F2EEC31F09BEC31F02AC182F495
:105350000401300E822796EC0EF02BC182F404017A
:10536000300E822796EC0EF02CC182F40401300E30
:10537000822796EC0EF02DC182F40401300E8227B4
:1053800096EC0EF02EC182F40401300E822796ECCA
:105390000EF02FC182F40401300E822796EC0EF03D
:1053A00030C182F40401300E822796EC0EF0040125
:1053B0002E0E826F96EC0EF031C182F40401300E95
:1053C000822796EC0EF032C182F40401300E82275F
:1053D00096EC0EF033C182F40401300E822796EC75
:1053E0000EF00401730E826F96EC0EF004012C0E89
:1053F000826F96EC0EF012EC32F059C100F15AC1F6
:1054000001F13FEC2CF013A255EF2AF004012C0E11
:10541000826F96EC0EF086C166F187C167F188C194
:1054200068F189C169F1ECEC22F00101000E046F12
:10543000000E056F010E066F000E076F2EEC31F0A7
:105440009BEC31F029672AEF2AF00401200E826FCD
:105450002DEF2AF004012D0E826F96EC0EF030C174
:1054600082F40401300E822796EC0EF031C182F4F2
:105470000401300E822796EC0EF004012E0E826F8E
:1054800096EC0EF032C182F40401300E822796ECC5
:105490000EF033C182F40401300E822796EC0EF038
:1054A00004016D0E826F96EC0EF003018351460AE3
:1054B00001E007D004012C0E826F96EC0EF0D4ECC4
:1054C00024F013A488EF2AF004012C0E826F96ECCE
:1054D0000EF013AC76EF2AF00401500E826F96ECBA
:1054E0000EF0139C1398139A88EF2AF013AE83EFF3
:1054F0002AF00401460E826F96EC0EF0139E13986C
:10550000139A88EF2AF00401530E826F96EC0EF086
:1055100037B09FEF2AF004012C0E826F96EC0EF04C
:105520008BB09AEF2AF00401440E826F96EC0EF0D5
:105530009FEF2AF00401530E826F96EC0EF00FB22B
:10554000A5EF2AF00FA0D7EF2AF004012C0E826FEE
:1055500096EC0EF0200EF86EF76AF66A0401090068
:10556000F5CF82F496EC0EF00900F5CF82F496ECBC
:105570000EF00900F5CF82F496EC0EF00900F5CF9D
:1055800082F496EC0EF00900F5CF82F496EC0EF062
:105590000900F5CF82F496EC0EF00900F5CF82F405
:1055A00096EC0EF00900F5CF82F496EC0EF0A0EC2C
:1055B0000EF00F90109E129815EF2BF00401630E61
:1055C000826F96EC0EF004012C0E826F96EC0EF0BA
:1055D0001BEC2BF004012C0E826F96EC0EF08EEC7F
:1055E0002BF004012C0E826F96EC0EF00AEC2CF0DE
:1055F00004012C0E826F96EC0EF00101F80E006F84
:10560000CD0E016F660E026F030E036F30EC2BF0B0
:1056100004012C0E826F96EC0EF020EC2CF0A0EC26
:105620000EF015EF2BF0A0EC0EF00301C26B07900B
:10563000109224EF2EF0D8900E0E64EC0BF0E8CF11
:1056400000F10F0E64EC0BF0E8CF01F1100E64ECEA
:105650000BF0E8CF02F1110E64EC0BF0E8CF03F190
:105660000101000E046F000E056F010E066F000EA3
:10567000076F2EEC31F09BEC31F02AC182F404016B
:10568000300E822796EC0EF02BC182F40401300E0E
:10569000822796EC0EF02CC182F40401300E822792
:1056A00096EC0EF02DC182F40401300E822796ECA8
:1056B0000EF02EC182F40401300E822796EC0EF01B
:1056C0002FC182F40401300E822796EC0EF030C117
:1056D00082F40401300E822796EC0EF031C182F480
:1056E0000401300E822796EC0EF004012E0E826F1C
:1056F00096EC0EF032C182F40401300E822796EC53
:105700000EF033C182F40401300E822796EC0EF0C5
:1057100004016D0E826F96EC0EF01200120E64EC16
:105720000BF0E8CF00F1130E64EC0BF0E8CF01F1C1
:10573000140E64EC0BF0E8CF02F1150E64EC0BF0E4
:10574000E8CF03F101010A0E046F000E056F000E91
:10575000066F000E076F0EEC31F0000E046F120E94
:10576000056F000E066F000E076F2EEC31F09BECFC
:1057700031F02AC182F40401300E822796EC0EF03B
:105780002BC182F40401300E822796EC0EF02CC15E
:1057900082F40401300E822796EC0EF02DC182F4C3
:1057A0000401300E822796EC0EF02EC182F4040123
:1057B000300E822796EC0EF02FC182F40401300ED9
:1057C000822796EC0EF030C182F40401300E82275D
:1057D00096EC0EF004012E0E826F96EC0EF031C1A5
:1057E00082F40401300E822796EC0EF032C182F46E
:1057F0000401300E822796EC0EF033C182F40401CE
:10580000300E822796EC0EF00401730E826F96EC38
:105810000EF012000A0E64EC0BF0E8CF00F10B0E54
:1058200064EC0BF0E8CF01F10C0E64EC0BF0E8CF68
:1058300002F10D0E64EC0BF0E8CF03F13FEF2CF01A
:10584000060E64EC0BF0E8CF00F1070E64EC0BF0F1
:10585000E8CF01F1080E64EC0BF0E8CF02F1090E7D
:1058600064EC0BF0E8CF03F13FEF2CF0010112ECF8
:1058700032F0078457C100F158C101F107940101CA
:10588000E80E046F800E056F000E066F000E076FA6
:105890000EEC31F0000E046F040E056F000E066F63
:1058A000000E076F2EEC31F0880E046F130E056F9B
:1058B000000E066F000E076FFDEC30F00A0E046F4D
:1058C000000E056F000E066F000E076F2EEC31F014
:1058D0009BEC31F00101296773EF2CF00401200EDD
:1058E000826F76EF2CF004012D0E826F96EC0EF095
:1058F00030C182F40401300E822796EC0EF031C1E3
:1059000082F40401300E822796EC0EF032C182F44C
:105910000401300E822796EC0EF004012E0E826FE9
:1059200096EC0EF033C182F40401300E822796EC1F
:105930000EF00401430E826F96EC0EF0120087C346
:105940002AF188C32BF189C32CF18AC32DF18BC3B3
:105950002EF18CC32FF18DC330F18EC331F190C382
:1059600032F191C333F10101296B60EC32F0D7ECD5
:1059700031F00101000E046F000E056F010E066F7D
:10598000000E076F0EEC31F00E0E0C6E00C10BF026
:105990004DEC0BF00F0E0C6E01C10BF04DEC0BF04B
:1059A000100E0C6E02C10BF04DEC0BF0110E0C6ED4
:1059B00003C10BF04DEC0BF004017A0E826F96ECF4
:1059C0000EF004012C0E826F96EC0EF00401350EE1
:1059D000826F96EC0EF004012C0E826F96EC0EF0A6
:1059E0001BEC2BF0C2EF22F087C32AF188C32BF106
:1059F00089C32CF18AC32DF18BC32EF18CC32FF1F7
:105A00008DC330F18EC331F190C332F191C333F1C4
:105A10000101296B60EC32F0D7EC31F0880E046F95
:105A2000130E056F000E066F000E076F02EC31F0CB
:105A3000000E046F040E056F000E066F000E076F58
:105A40000EEC31F00101E80E046F800E056F000EC0
:105A5000066F000E076F2EEC31F00A0E0C6E00C1BF
:105A60000BF04DEC0BF00B0E0C6E01C10BF04DEC7E
:105A70000BF00C0E0C6E02C10BF04DEC0BF00D0E8A
:105A80000C6E03C10BF04DEC0BF004017A0E826F2B
:105A900096EC0EF004012C0E826F96EC0EF00401D1
:105AA000360E826F96EC0EF004012C0E826F96EC8F
:105AB0000EF00AEC2CF0C2EF22F087C32AF188C363
:105AC0002BF189C32CF18AC32DF18BC32EF18CC32A
:105AD0002FF18DC330F18FC331F190C332F191C3F7
:105AE00033F1010160EC32F0D7EC31F0000E046FBD
:105AF000120E056F000E066F000E076F0EEC31F0F0
:105B000001010A0E046F000E056F000E066F000EF5
:105B1000076F2EEC31F0120E0C6E00C10BF04DEC45
:105B20000BF0130E0C6E01C10BF04DEC0BF0140ECC
:105B30000C6E02C10BF04DEC0BF0150E0C6E03C198
:105B40000BF04DEC0BF004017A0E826F96EC0EF028
:105B500004012C0E826F96EC0EF00401370E826F5A
:105B600096EC0EF004012C0E826F96EC0EF08EEC8B
:105B70002BF0C2EF22F087C32AF188C32BF189C32F
:105B80002CF18AC32DF18BC32EF18CC32FF18DC361
:105B900030F18EC331F190C332F191C333F1010181
:105BA000296B60EC32F0D7EC31F0880E046F130EE5
:105BB000056F000E066F000E076F02EC31F0000E4D
:105BC000046F040E056F000E066F000E076F0EECDB
:105BD00031F00101E80E046F800E056F000E066FB4
:105BE000000E076F2EEC31F0060E0C6E00C10BF0AC
:105BF0004DEC0BF0070E0C6E01C10BF04DEC0BF0F1
:105C0000080E0C6E02C10BF04DEC0BF0090E0C6E81
:105C100003C10BF04DEC0BF004017A0E826F96EC91
:105C20000EF004012C0E826F96EC0EF00401380E7B
:105C3000826F96EC0EF004012C0E826F96EC0EF043
:105C400020EC2CF0C2EF22F007A897EF2EF0010114
:105C5000800E006F1A0E016F060E026F000E036FAA
:105C60004BC104F14CC105F14DC106F14EC107F124
:105C7000FDEC30F003BFDDEF2EF058EC2FF04BC100
:105C800000F14CC101F14DC102F14EC103F1078297
:105C90000AEC30F018C104F119C105F11AC106F17E
:105CA0001BC107F1F80E006FCD0E016F660E026F7B
:105CB000030E036FFDEC30F00E0E0C6E00C10BF006
:105CC0004DEC0BF00F0E0C6E01C10BF04DEC0BF018
:105CD000100E0C6E02C10BF04DEC0BF0110E0C6EA1
:105CE00003C10BF04DEC0BF00784010112EC32F014
:105CF00057C100F158C101F107940A0E0C6E00C1A2
:105D00000BF04DEC0BF00B0E0C6E01C10BF04DECDB
:105D10000BF00C0E0C6E02C10BF04DEC0BF00D0EE7
:105D20000C6E03C10BF04DEC0BF0DDEF2EF007AA6B
:105D3000DDEF2EF00784010112EC32F057C100F1C3
:105D400058C101F10794060E0C6E00C10BF04DEC2A
:105D50000BF0070E0C6E01C10BF04DEC0BF0080EB2
:105D60000C6E02C10BF04DEC0BF0090E0C6E03C172
:105D70000BF04DEC0BF0078462C100F163C101F13F
:105D800064C102F165C103F10794120E0C6E00C1EB
:105D90000BF04DEC0BF0130E0C6E01C10BF04DEC43
:105DA0000BF0140E0C6E02C10BF04DEC0BF0150E47
:105DB0000C6E03C10BF04DEC0BF00798079A040131
:105DC000805181197F0B0DE09EA8FED714EE00F0E4
:105DD00081517F0BE126E750812B0F01AD6EDFEF84
:105DE0002EF005012F51000AD8B420EF2FF081BA10
:105DF00005EF2FF015B220EF2FF005012F51010A0A
:105E0000D8B41EEF2FF017EF2FF005012F51000A25
:105E1000D8B4D7EF39F005012F51010AD8B41EEFDD
:105E20002FF000011650050AD8B4D7EF39F081B829
:105E300020EF2FF05BEC33F059EC34F070EC39F0DC
:105E4000C4EF0DF018C100F119C101F11AC102F13E
:105E50001BC103F1000E046F000E056F010E066FEB
:105E6000000E076F2EEC31F029A14DEF2FF02051DD
:105E7000D8B44DEF2FF018C100F119C101F11AC1CA
:105E800002F11BC103F1000E046F000E056F0A0E34
:105E9000066F000E076F2EEC31F012000101045165
:105EA0000013055101130651021307510313120089
:105EB0000101186B196B1A6B1B6B12002AC182F45B
:105EC0000401300E822796EC0EF02BC182F40401FF
:105ED000300E822796EC0EF02CC182F40401300EB5
:105EE000822796EC0EF02DC182F40401300E822739
:105EF00096EC0EF02EC182F40401300E822796EC4F
:105F00000EF02FC182F40401300E822796EC0EF0C1
:105F100030C182F40401300E822796EC0EF031C1BC
:105F200082F40401300E822796EC0EF032C182F426
:105F30000401300E822796EC0EF033C182F4040186
:105F4000300E822796EC0EF012002FC182F404016D
:105F5000300E822796EC0EF030C182F40401300E30
:105F6000822796EC0EF031C182F40401300E8227B4
:105F700096EC0EF032C182F40401300E822796ECCA
:105F80000EF033C182F40401300E822796EC0EF03D
:105F90001200060E216E060E226E060E236E212EB4
:105FA000CFEF2FF0222ECFEF2FF0232ECFEF2FF0B9
:105FB0008B84020E216E020E226E020E236E212EA3
:105FC000DFEF2FF0222EDFEF2FF0232EDFEF2FF069
:105FD0008B941200FF0E226E22C023F0030E216E5E
:105FE0008B84212EF0EF2FF0030E216E232EF0EF85
:105FF0002FF08B9422C023F0030E216E212EFEEF92
:106000002FF0030E216E233EFEEF2FF0222EECEF39
:106010002FF012000101005305E1015303E1025387
:1060200001E1002BCDEC30F012EC32F03951006F71
:106030003A51016F420E046F4B0E056F000E066F52
:10604000000E076F0EEC31F000C104F101C105F143
:1060500002C106F103C107F118C100F119C101F134
:106060001AC102F11BC103F107B23BEF30F002ECA1
:1060700031F03DEF30F0FDEC30F000C118F101C11E
:1060800019F102C11AF103C11BF1120012EC32F036
:1060900059C100F15AC101F1060E64EC0BF0E8CFD2
:1060A00004F1070E64EC0BF0E8CF05F1080E64EC88
:1060B0000BF0E8CF06F1090E64EC0BF0E8CF07F126
:1060C000FDEC30F000C124F101C125F102C126F13F
:1060D00003C127F1290E046F000E056F000E066F35
:1060E000000E076F0EEC31F0EE0E046F430E056FDD
:1060F000000E066F000E076F02EC31F024C104F1B0
:1061000025C105F126C106F127C107F10EEC31F0DA
:1061100000C11CF101C11DF102C11EF103C11FF13B
:10612000120E64EC0BF0E8CF04F1130E64EC0BF0EC
:10613000E8CF05F1140E64EC0BF0E8CF06F1150E74
:1061400064EC0BF0E8CF07F10D0E006F000E016F4D
:10615000000E026F000E036F0EEC31F0180E046F8C
:10616000000E056F000E066F000E076F2EEC31F06B
:106170001CC104F11DC105F11EC106F11FC107F1CB
:1061800002EC31F06A0E046F2A0E056F000E066FE6
:10619000000E076FFDEC30F01200BF0EFA6E200EFD
:1061A0003A6F396BD8900037013702370337D8B0D0
:1061B000DEEF30F03A2FD3EF30F039073A070353D0
:1061C000D8B412000331070B80093F6F03390F0B5E
:1061D000010F396F80EC5FF0406F390580EC5FF0A4
:1061E000405D405F396B3F33D8B0392739333FA921
:1061F000F3EF30F0405139271200010137EC32F053
:10620000D8B01200010103510719346FFAEC31F0D4
:10621000D8900751031934AF800F12000101346B7D
:106220001EEC32F0D8A034EC32F0D8B0120009ECF9
:1062300032F012EC32F01F0E366F4AEC32F00B35B2
:10624000D8B0FAEC31F0D8A00335D8B01200362F10
:106250001DEF31F034B121EC32F012000101346B4A
:1062600004510511061107110008D8A01EEC32F0E8
:10627000D8A034EC32F0D8B01200086B096B0A6B6E
:106280000B6B4AEC32F01F0E366F4AEC32F00751BE
:106290000B5DD8A458EF31F006510A5DD8A458EF31
:1062A00031F00551095DD8A458EF31F00451085D73
:1062B000D8A06BEF31F00451085F0551D8A0053D1F
:1062C000095F0651D8A0063D0A5F0751D8A0073DD7
:1062D0000B5FD8900081362F45EF31F034B121ECBF
:1062E00032F0346B1EEC32F0D8904EEC32F00751A5
:1062F0000B5DD8A488EF31F006510A5DD8A488EF71
:1063000031F00551095DD8A488EF31F00451085DE2
:10631000D8A097EF31F0003F97EF31F0013F97EFB2
:1063200031F0023F97EF31F0032BD8B4120034B1B3
:1063300021EC32F012000101346B1EEC32F0D8B0C7
:10634000120053EC32F0200E366F0037013702375F
:10635000033711EE33F00A0E376FE7360A0EE75CAB
:10636000D8B0E76EE552372FADEF31F0362FA5EFFD
:1063700031F034B12981D890120053EC32F0200E64
:10638000366F003701370237033711EE33F00A0E4C
:10639000376FE7360A0EE75CD8B0E76EE552372F65
:1063A000C9EF31F0362FC1EF31F0D8901200010162
:1063B0000A0E346F200E366F11EE29F03451376F0C
:1063C0000A0ED890E652D8B0E726E732372FE2EF30
:1063D00031F00333023301330033362FDCEF31F079
:1063E000E750FF0FD8A00335D8B0120029B121EC37
:1063F00032F01200045100270551D8B0053D0127A5
:106400000651D8B0063D02270751D8B0073D0327F3
:1064100012000051086F0151096F02510A6F0351B8
:106420000B6F12000101006B016B026B036B12001A
:106430000101046B056B066B076B12000335D8A0D6
:1064400012000351800B001F011F021F031F003F9A
:1064500031EF32F0013F31EF32F0023F31EF32F0F5
:10646000032B342B032512000735D8A01200075147
:10647000800B041F051F061F071F043F47EF32F064
:10648000053F47EF32F0063F47EF32F0072B342B42
:10649000072512000037013702370337083709375D
:1064A0000A370B3712000101296B2A6B2B6B2C6BFF
:1064B0002D6B2E6B2F6B306B316B326B336B12008D
:1064C00001012A510F0B2A6F2B510F0B2B6F2C51EF
:1064D0000F0B2C6F2D510F0B2D6F2E510F0B2E6F9D
:1064E0002F510F0B2F6F30510F0B306F31510F0B9E
:1064F000316F32510F0B326F33510F0B336F12006C
:1065000000C124F101C125F102C126F103C127F127
:1065100004C100F105C101F106C102F107C103F197
:1065200024C104F125C105F126C106F127C107F1F7
:10653000120010A806D08994000EC76E220EC66EF7
:1065400005D08984000EC76E220EC66E050EE82E99
:10655000FED7120010A802D0898401D08994050EBC
:10656000E82EFED7120099EC32F09E96C69E000EE1
:10657000C96EFF0E9EB602D0E82EFCD79E96C69E30
:10658000000EC96EFF0E9EB602D0E82EFCD7C9CF12
:10659000AFF59E96C69E000EC96EFF0E9EB602D047
:1065A000E82EFCD7C9CFB0F59E96C69E000EC96EE8
:1065B000FF0E9EB602D0E82EFCD7C9CFB1F59E964D
:1065C000C69E000EC96EFF0E9EB602D0E82EFCD706
:1065D000C9CFB2F59E96C69E000EC96EFF0E9EB63E
:1065E00002D0E82EFCD7C9CFB3F59E96C69E000E0A
:1065F000C96EFF0E9EB602D0E82EFCD7C9CFB4F507
:106600009E96C69E000EC96EFF0E9EB602D0E82E64
:10661000FCD7C9CFB5F5AAEC32F0120099EC32F0F4
:106620009E96C69E800EC96EFF0E9EB602D0E82EC4
:10663000FCD79E96C69EAFC5C9FFFF0E9EB602D080
:10664000E82EFCD79E96C69EB0C5C9FFFF0E9EB62B
:1066500002D0E82EFCD79E96C69EB1C5C9FFFF0E9C
:106660009EB602D0E82EFCD79E96C69EB2C5C9FF44
:10667000FF0E9EB602D0E82EFCD79E96C69EB3C5EE
:10668000C9FFFF0E9EB602D0E82EFCD79E96C69E8E
:10669000B4C5C9FFFF0E9EB602D0E82EFCD79E9669
:1066A000C69EB5C5C9FFFF0E9EB602D0E82EFCD728
:1066B000AAEC32F0120099EC32F09E96C69E070EBC
:1066C000C96EFF0E9EB602D0E82EFCD79E96C69EDF
:1066D000000EC96EFF0E9EB602D0E82EFCD7C9CFC1
:1066E000AFF59E96C69E000EC96EFF0E9EB602D0F6
:1066F000E82EFCD7C9CFB0F59E96C69E000EC96E97
:10670000FF0E9EB602D0E82EFCD7C9CFB1F59E96FB
:10671000C69E000EC96EFF0E9EB602D0E82EFCD7B4
:10672000C9CFB2F5AAEC32F099EC32F09E96C69E33
:1067300025C0C9FFFF0E9EB602D0E82EFCD79E965C
:10674000C69E000EC96EFF0E9EB602D0E82EFCD784
:10675000C9CFB6F5AAEC32F0120099EC32F09E9651
:10676000C69E870EC96EFF0E9EB602D0E82EFCD7DD
:106770009E96C69EAFC5C9FFFF0E9EB602D0E82EFC
:10678000FCD79E96C69EB0C5C9FFFF0E9EB602D02E
:10679000E82EFCD79E96C69EB1C5C9FFFF0E9EB6D9
:1067A00002D0E82EFCD79E96C69EB2C5C9FFFF0E4A
:1067B0009EB602D0E82EFCD7AAEC32F099EC32F06B
:1067C0009E96C69E26C0C9FFFF0E9EB602D0E82E3A
:1067D000FCD79E96C69EB6C5C9FFFF0E9EB602D0D8
:1067E000E82EFCD7AAEC32F0120099EC32F09E961B
:1067F000C69E870EC96EFF0E9EB602D0E82EFCD74D
:106800009E96C69E000EC96EFF0E9EB602D0E82E62
:10681000FCD79E96C69E800EC96EFF0E9EB602D015
:10682000E82EFCD79E96C69E800EC96EFF0E9EB6C1
:1068300002D0E82EFCD79E96C69E800EC96EFF0E33
:106840009EB602D0E82EFCD7AAEC32F0120099ECEA
:1068500032F09E96C69E870EC96EFF0E9EB602D07F
:10686000E82EFCD79E96C69E000EC96EFF0E9EB601
:1068700002D0E82EFCD79E96C69E000EC96EFF0E73
:106880009EB602D0E82EFCD79E96C69E800EC96E9C
:10689000FF0E9EB602D0E82EFCD79E96C69E800EB6
:1068A000C96EFF0E9EB602D0E82EFCD7AAEC32F0DD
:1068B000120010A817D099EC32F09E96C69E8F0E4B
:1068C000C96EFF0E9EB602D0E82EFCD79E96C69EDD
:1068D000000EC96EFF0E9EB602D0E82EFCD7AAECC1
:1068E00032F012005BEC33F0120010A82DD099ECBE
:1068F00032F09E96C69E26C0C9FFFF0E9EB602D0FD
:10690000E82EFCD79E96C69E450EC96EFF0E9EB61B
:1069100002D0E82EFCD7AAEC32F099EC32F09E9629
:10692000C69E8F0EC96EFF0E9EB602D0E82EFCD713
:106930009E96C69E000EC96EFF0E9EB602D0E82E31
:10694000FCD7AAEC32F0120099EC32F09E96C69E6B
:1069500026C0C9FFFF0E9EB602D0E82EFCD79E9639
:10696000C69E010EC96EFF0E9EB602D0E82EFCD761
:10697000AAEC32F099EC32F09E96C69E910EC96E4A
:10698000FF0E9EB602D0E82EFCD79E96C69EA50EA0
:10699000C96EFF0E9EB602D0E82EFCD7AAEC32F0EC
:1069A000120099EC32F09E96C69E26C0C9FFFF0EDB
:1069B0009EB602D0E82EFCD79E96C69E810EC96E6A
:1069C000FF0E9EB602D0E82EFCD7AAEC32F01200E1
:1069D00099EC32F09E96C69E26C0C9FFFF0E9EB669
:1069E00002D0E82EFCD79E96C69E010EC96EFF0E01
:1069F0009EB602D0E82EFCD7AAEC32F0120099EC39
:106A000032F09E96C69E910EC96EFF0E9EB602D0C3
:106A1000E82EFCD79E96C69EA50EC96EFF0E9EB6AA
:106A200002D0E82EFCD7AAEC32F0120099EC32F03A
:106A30009E96C69E910EC96EFF0E9EB602D0E82E9F
:106A4000FCD79E96C69E000EC96EFF0E9EB602D063
:106A5000E82EFCD7AAEC32F012000501256B266B5C
:106A6000276B286B899A400EC76E200EC66E9E96C5
:106A7000C69E030EC96EFF0E9EB602D0E82EFCD74E
:106A80009E96C69E27C5C9FFFF0E9EB602D0E82E71
:106A9000FCD79E96C69E26C5C9FFFF0E9EB602D0A5
:106AA000E82EFCD79E96C69E25C5C9FFFF0E9EB652
:106AB00002D0E82EFCD79E96C69EC952FF0E9EB607
:106AC00002D0E82EFCD7898A0F01C950FF0A01E1E4
:106AD000120005012E51130A05E005012E51170A77
:106AE0000CE012000501E00E256FFF0E266F0F0E61
:106AF000276F000E286F86EF35F00501E00E256F39
:106B0000FF0E266FFF0E276F000E286F899A400E2A
:106B1000C76E200EC66E9E96C69E030EC96EFF0EF1
:106B20009EB602D0E82EFCD79E96C69E27C5C9FF0A
:106B3000FF0E9EB602D0E82EFCD79E96C69E26C5B6
:106B4000C9FFFF0E9EB602D0E82EFCD79E96C69EC9
:106B500025C5C9FFFF0E9EB602D0E82EFCD79E9633
:106B6000C69EC952FF0E9EB602D0E82EFCD7898A77
:106B70000F01C950FF0A1DE005012E51130A05E05F
:106B800005012E51170A0BE012000501000E256FBA
:106B9000000E266F100E276F000E286F12000501E1
:106BA000000E256F000E266F000E276F010E286F56
:106BB00012000501256B266B276B286B05012E51F2
:106BC000130A05E005012E51170A0CE01200050119
:106BD000000E216F000E226F080E236F000E246F2F
:106BE000FBEF35F00501000E216F000E226F800EC5
:106BF000236F000E246F21C500F122C501F123C5CA
:106C000002F124C503F125C504F126C505F127C508
:106C100006F128C507F14EEC2FF000C125F501C1A2
:106C200026F502C127F503C128F5899A400EC76EE3
:106C3000200EC66E9E96C69E030EC96EFF0E9EB6B1
:106C400002D0E82EFCD79E96C69E27C5C9FFFF0E30
:106C50009EB602D0E82EFCD79E96C69E26C5C9FFDA
:106C6000FF0E9EB602D0E82EFCD79E96C69E25C586
:106C7000C9FFFF0E9EB602D0E82EFCD79E96C69E98
:106C8000C952FF0E9EB602D0E82EFCD7898AC950A1
:106C9000FF0A08E104C125F505C126F506C127F55F
:106CA00007C128F5D890050124332333223321333B
:106CB0002151E00B216F0501216766EF36F0226755
:106CC00066EF36F0236766EF36F02467FBEF35F0AA
:106CD0000501200E2527E86A2623E86A2723E86AAB
:106CE00028231200E86A05012E51130A06E0050167
:106CF0002E51170A0BE0020E120005012851000A5E
:106D000003E12751F00B07E0010E120005012851A5
:106D1000000A01E0010E120029C500F12AC501F1A7
:106D20002BC502F12CC503F125C504F126C505F1DB
:106D300027C506F128C507F1FDEC30F003BF1200AE
:106D400072EC36F0D8A404EF37F0899A400EC76E83
:106D5000200EC66E9E96C69E060EC96EFF0E9EB68D
:106D600002D0E82EFCD7898A899A9E96C69E020E8A
:106D7000C96EFF0E9EB602D0E82EFCD79E96C69E28
:106D800027C5C9FFFF0E9EB602D0E82EFCD79E96FF
:106D9000C69E26C5C9FFFF0E9EB602D0E82EFCD7C0
:106DA0009E96C69E25C5C9FFFF0E9EB602D0E82E50
:106DB000FCD79E96C69E000EC96EFF0E9EB602D0F0
:106DC000E82EFCD7898A899A9E96C69E050EC96EC2
:106DD000FF0E9EB602D0E82EFCD79E96C69EC952E4
:106DE000FF0E9EB602D0E82EFCD7C9B0EDEF36F00C
:106DF000898A0501200E2527E86A2623E86A2723C9
:106E0000E86A28238CEF36F01200899A400EC76E8C
:106E1000200EC66E9E96C69E060EC96EFF0E9EB6CC
:106E200002D0E82EFCD7898A899A9E96C69EC70E04
:106E3000C96EFF0E9EB602D0E82EFCD7898A0501E6
:106E4000256B266B276B286B1200899A400EC76E44
:106E5000200EC66E9E96C69E050EC96EFF0E9EB68D
:106E600002D0E82EFCD79E96C69EC952FF0E9EB653
:106E700002D0E82EFCD7C9CF37F5898A1200899A4B
:106E8000400EC76E200EC66E9E96C69EB90EC96E87
:106E9000FF0E9EB602D0E82EFCD7898A1200899A8E
:106EA000400EC76E200EC66E9E96C69EAB0EC96E75
:106EB000FF0E9EB602D0E82EFCD7898AFF0EE82E80
:106EC000FED7120072EC36F0D8A41200899A400E58
:106ED000C76E200EC66E9E96C69E030EC96EFF0E2E
:106EE0009EB602D0E82EFCD79E96C69E27C5C9FF47
:106EF000FF0E9EB602D0E82EFCD79E96C69E26C5F3
:106F0000C9FFFF0E9EB602D0E82EFCD79E96C69E05
:106F100025C5C9FFFF0E9EB602D0E82EFCD79E966F
:106F2000C69EC952FF0E9EB602D0E82EFCD7898AB3
:106F30000F01C950FF0AD8A4E1EF38F00501FE0E99
:106F4000376F0501FF0E536FFF0E546FFF0E556F25
:106F5000FF0E566F15A637991586B3EC32F0AFC504
:106F600038F5B0C539F5B1C53AF5B2C53BF5B3C58D
:106F70003CF5B4C53DF5B5C53EF50784BAC166F12B
:106F8000BBC167F1BCC168F1BDC169F14BC14FF133
:106F90004CC150F14DC151F14EC152F157C159F19F
:106FA00058C15AF100011650010AD8B4E6EF37F083
:106FB00000011650020AD8B40BEF38F00001165049
:106FC000040AD8B430EF38F0E1EF38F00501476B30
:106FD000486B496B4A6B05014B6B4C6B4D6B4E6BB1
:106FE00005014F6B506B516B526B8BA0379BECECD8
:106FF00022F000C1DAF101C1DBF102C1DCF103C111
:10700000DDF100C13FF501C140F502C141F503C109
:1070100042F54FEF38F00501476B486B496B4A6BFF
:1070200005014B6B4C6B4D6B4E6B05014F6B506B01
:10703000516B526BECEC22F000C1DAF101C1DBF1D3
:1070400002C1DCF103C1DDF1E9EC23F000C147F539
:1070500001C148F502C149F503C14AF5E1EF38F035
:10706000379BDAC13FF5DBC140F5DCC141F5DDC13D
:1070700042F5ECEC22F000C14BF501C14CF502C128
:107080004DF503C14EF5E9EC23F000C14FF501C108
:1070900050F502C151F503C152F54FEF38F005012B
:1070A00061675AEF38F062675AEF38F063675AEF5A
:1070B00038F064675EEF38F073EF38F0DAC100F152
:1070C000DBC101F1DCC102F1DDC103F161C504F1F5
:1070D00062C505F163C506F164C507F1FDEC30F04A
:1070E00003BFE1EF38F059C143F55AC144F5B9C5C2
:1070F00045F50501210E326F899A400EC76E200EAC
:10710000C66E9E96C69E060EC96EFF0E9EB602D035
:10711000E82EFCD7898A899A9E96C69E020EC96E71
:10712000FF0E9EB602D0E82EFCD79E96C69E27C5BF
:10713000C9FFFF0E9EB602D0E82EFCD79E96C69ED3
:1071400026C5C9FFFF0E9EB602D0E82EFCD79E963C
:10715000C69E25C5C9FFFF0E9EB602D0E82EFCD7FD
:1071600025EE37F0322F02D0C1EF38F09E96C69E42
:10717000DECFC9FFFF0E9EB602D0E82EFCD7B2EFDD
:1071800038F0898A899A9E96C69E050EC96EFF0EB2
:107190009EB602D0E82EFCD79E96C69EC952FF0E20
:1071A0009EB602D0E82EFCD7C9B0CCEF38F0898A61
:1071B0000501200E2527E86A2623E86A2723E86AC6
:1071C000282315900794120021C500F122C501F172
:1071D00023C502F124C503F1899A400EC76E200E23
:1071E000C66E9E96C69E0B0EC96EFF0E9EB602D050
:1071F000E82EFCD79E96C69E02C1C9FFFF0E9EB622
:1072000002D0E82EFCD79E96C69E01C1C9FFFF0E94
:107210009EB602D0E82EFCD79E96C69E00C1C9FF3E
:10722000FF0E9EB602D0E82EFCD79E96C69EC9528F
:10723000FF0E9EB602D0E82EFCD725EE37F00501F2
:10724000200E326F9E96C69EC952FF0E9EB602D089
:10725000E82EFCD7C9CFDEFF322F22EF39F0898A22
:107260001200899A400EC76E200EC66E9E96C69E6C
:10727000900EC96EFF0E9EB602D0E82EFCD79E96E9
:10728000C69E000EC96EFF0E9EB602D0E82EFCD739
:107290009E96C69E000EC96EFF0E9EB602D0E82EC8
:1072A000FCD79E96C69E000EC96EFF0E9EB602D0FB
:1072B000E82EFCD79E96C69EC952FF0E9EB602D0FF
:1072C000E82EFCD7C9CF2DF59E96C69EC952FF0E5B
:1072D0009EB602D0E82EFCD7C9CF2EF5898A1200BF
:1072E000B3EC32F005012F51010A5FE005012F5187
:1072F000020A16E005012F51030A19E005012F517A
:10730000040A24E005012F51050A2BE005012F5145
:10731000060A39E005012F51070A3FE0D5EF39F0A1
:10732000602FD3EF39F05FC560F5D5EF39F0B0C508
:1073300000F101010F0E001701010051000A35E0B4
:1073400001010051050A31E0D3EF39F0B0C500F179
:1073500001010F0E001701010051000A26E0D3EFD2
:1073600039F00501B051000A20E00501B051150ABD
:107370001CE00501B051300A18E00501B051450A82
:1073800014E0D3EF39F00501B051000A0EE0050119
:10739000B051300A0AE0D3EF39F00501B051000ACC
:1073A00004E0D3EF39F015901200158012008B9095
:1073B000C9EC2FF0B9C5E8FFD70802E3C9EC2FF0FC
:1073C000B9C5E8FFC80802E3C9EC2FF0B9C5E8FF6A
:1073D000B90802E3C9EC2FF0B9C5E8FFAA0802E337
:1073E000C9EC2FF0B9C5E8FF9B0802E3C9EC2FF008
:1073F0003FEC37F0F29CF29E8B94C69AC290948236
:10740000948C720ED36ED3A4FED789968A909390F3
:10741000F29AF2949D909E909D929E92F298F29292
:1074200059EC34F0FF0EE8CF00F0E82EFED7002E26
:10743000FCD7F290F286815081A821EF3AF0F29EBB
:107440000300700ED36EF296F29015840380EAEC7E
:067450002FF09AEF0BF093
:10BF0000E844F926000C160C2B0C3F0C520C640C68
:10BF1000760C860C960CA50CB30CC10CCF0CDC0C6B
:06BF2000E80CF40C000C1B
:0200000400F00A
:0100C800FE39
:00000001FF
